:020000040800F2
:1030000018190020C9310008F7980008954F0008EA
:10301000F5980008713800087BAC0008000000003B
:1030200000000000000000000000000095A3000860
:103030003742000800000000ADA000089DA600086F
:10304000E3310008E3310008E3310008E331000810
:10305000E3310008E3310008E3310008E331000800
:10306000E3310008E3310008E3310008B94000080B
:10307000E3310008E3310008E3310008E3310008E0
:10308000E3310008E331000801350008E3310008AE
:10309000CDAB0008E3310008E3310008E33100085C
:1030A000E9A6000839A70008E3310008E331000869
:1030B00081A70008E3310008C9A70008E331000830
:1030C000E3310008E3310008E3310008E331000890
:1030D000E331000869AB00086DAB0008E33100087C
:1030E000E3310008E3310008E331000800F002F8A2
:1030F00000F05AF80AA090E8000C82448344AAF138
:103100000107DA4501D100F04FF8AFF2090EBAE835
:103110000F0013F0010F18BFFB1A43F0010318470B
:10312000589B0000789B00000A444FF0000C10F8F8
:10313000013B13F0070408BF10F8014B1D1108BF35
:1031400010F8015B641E05D010F8016B641E01F8D5
:10315000016BF9D113F0080F1EBF10F8014BAD1C25
:103160000C1B09D16D1E58BF01F801CBFAD505E043
:1031700014F8016B01F8016B6D1EF9D59142D6D39D
:10318000704700000023002400250026103A28BFC5
:1031900078C1FBD8520728BF30C148BF0B607047C9
:1031A0001FB51FBD10B510BD00F070F91146FFF737
:1031B000F7FF08F099F800F08EF903B4FFF7F2FF7B
:1031C00003BC00F095F90000094880470948004712
:1031D000FEE7FEE7FEE7FEE7FEE7FEE7FEE7FEE7C7
:1031E000FEE7FEE704480549054A064B7047000024
:1031F000A9A60008ED3000081813002018190020B7
:10320000181500201815002053EA020C00F0698000
:103210002DE9F04B4FF00006002B1FBFB3FA83F5EA
:1032200003FA05F424FA05F65E4012BF1643B2FA1B
:1032300082F502FA05F4C5F120051EBF22FA05FC4D
:1032400044EA0C04203556EA044C4FEA144418BFF3
:10325000641C4FF000084FF00009904271EB030C22
:1032600039D3002919BFB1FA81F701FA07F6B0FA8C
:1032700080F700FA07F6C7F120071EBF20FA07FC07
:1032800046EA0C062037B6FBF4FCA7EB0507103F17
:1032900007F01F0BCBF120060CFA0BFB2CFA06F6FD
:1032A00044BFB3460026202FA4BF5E464FF0000B5C
:1032B0005BEA060C08BF4FF0010B19EB0B09ABFBE7
:1032C000027C48EB0608C01B06FB02CC0BFB03CCC0
:1032D00071EB0C01C1E70B46024641464846BDE88A
:1032E000F08B13B54FF000004FF00001AFF30080FA
:1032F000BDE81C407047032A40F2308010F0030CF8
:1033000000F0158011F8013BBCF1020F624498BF38
:1033100011F801CB00F8013B38BF11F8013BA2F1D5
:10332000040298BF00F801CB38BF00F8013B11F050
:10333000030300F05280083AC0F0088051F8043BC3
:10334000083A51F804CBA0E80810F5E7121D5CBF5D
:1033500051F8043B40F8043BAFF30080D20724BF90
:1033600011F8013B11F801CB48BF11F8012B24BF24
:1033700000F8013B00F801CB48BF00F8012B704773
:1033800002F0FF0343EA032242EA024200F002B8DD
:103390004FF000020429C0F0128010F0030C00F07E
:1033A0005080CCF1040CBCF1020F18BF00F8012BC7
:1033B000A8BF20F8022BA1EB0C0100F042B85FEA95
:1033C000C17C24BF00F8012B00F8012B48BF00F896
:1033D000012B704770477047704710B5203AC0F016
:1033E0000B80B1E81850203AA0E81850B1E8185006
:1033F000A0E81850BFF4F5AF5FEA027C24BFB1E843
:103400001850A0E8185044BF18C918C0BDE81040B3
:103410005FEA827C24BF51F8043B40F8043B08BFBC
:103420007047D20728BF31F8023B48BF11F8012B83
:1034300028BF20F8023B48BF00F8012B70474FF02F
:10344000000200B5134694469646203922BFA0E8F4
:103450000C50A0E80C50B1F12001BFF4F7AF090700
:1034600028BFA0E80C5048BF0CC05DF804EB8900F1
:1034700028BF40F8042B08BF704748BF20F8022B34
:1034800011F0804F18BF00F8012B7047754600F00F
:103490002BF8AE4605006946534620F007008546E6
:1034A00018B020B5FFF79EFEBDE820404FF00006A3
:1034B0004FF000074FF000084FF0000B21F007011C
:1034C000AC46ACE8C009ACE8C009ACE8C009ACE85F
:1034D000C0098D46704710B50446AFF30080204602
:1034E000BDE81040FFF769BE00487047B8120020E1
:1034F00001491820ABBEFEE726000200704700001D
:1035000004480168490704D56FF00401016005F023
:1035100022BE70470024014070B5114C02212046A4
:1035200000F024F802210F4800F020F8022000F0FB
:10353000CFFD0021204600F01AF90B4D002128464E
:1035400000F0D2FD084A0421083AD1600121284642
:1035500000F0CAFD2046BDE87040012100F007B927
:10356000002401400028014008000240C9430160D6
:1035700070470029816802D041F0010101E021F08B
:103580000101816070470029816802D041F4807197
:1035900001E021F480718160704700000D4910B591
:1035A000884202D1012144150AE00B49884202D128
:1035B0000121041504E0094988420AD10121CC0304
:1035C000204606F0AFFD2046BDE81040002106F081
:1035D000A9BD10BD0024014000280140003C01406D
:1035E0000029816802D041F4801101E021F48011AA
:1035F000816070470029816802D041F4004101E0F8
:1036000021F4004181607047826822F4E0420A435D
:103610008168914200D0826070470146002089682D
:10362000490700D5012070470246002012680A426F
:1036300000D00120704708B5084428300090006889
:1036400080B208BD002A4268C9B201D00A4300E036
:103650008A4342607047000010B542680E4B0C79F7
:103660001A400B6842EA04221343436082680B4B02
:103670001A40D1E9024323434C7942EA44021343FE
:103680008360C26A097C22F47002491EC9B242EA10
:103690000151C16210BD0000FFFEF0FFFDF7F1FF18
:1036A00070B5072609290AD9C568A1F10A0404EBF7
:1036B0004404A640B543A3401D43C56007E0056927
:1036C00001EB4104A640B543A3401D430561836B54
:1036D000C3F30154121B921C02EB82021F2494407C
:1036E000A34391400B43836370BD826B491E22F458
:1036F000401242EA01518163704770B507260929DB
:103700000AD9C568A1F10A0404EB4404A640B543F4
:10371000A3401D43C56007E0056901EB4104A640D5
:10372000B543A3401D4305611F23072A09D2446BFB
:10373000521E02EB820293409C4391400C4344632F
:1037400070BD0D2A09D2046BD21F02EB8202934096
:103750009C4391400C43046370BDC46A0D3A02EB74
:10376000820293409C4391400C43C46270BD002987
:10377000816802D041F4A00101E021F4A001816040
:1037800070470029816802D041F4021101E021F460
:10379000021181607047816841F0040181607047C7
:1037A00000210160017141718160C16001210174DA
:1037B0007047000070B5194A194C9088A18868B10B
:1037C000D38819448DB2174909780023012907D0FD
:1037D0005178142905D2491C517002E0918016E0FD
:1037E0005370854202D900F101000FE00FD20B485F
:1037F000517880881429A0F1010080B206D2117896
:10380000491CC9B21170052901D3137090809088AA
:1038100007F0A6FE08F08CFBE07070BD7C00002075
:103820006804002069020020F0B50F4D0F4C002104
:103830006E88AF8DA378084604F11402BE4201D908
:1038400022F8136032F81060401CC0B231441028D6
:10385000F8D30809A8805B1CD8B2A070102801D347
:103860000020A070F0BD0000200400209400002083
:10387000FEE70000F0B55E4944F278530C228878E8
:1038800038B301283ED045F20C1346F61044032805
:1038900051D045F6A04545F2E84646F2584705287E
:1038A00060D048F6F12C042871D006286ED00E8125
:1038B00046F6FE5048818C81CB8144F61E7008820A
:1038C0004D8241F2CC00888240F66E70C882494831
:1038D0002EE043F22C20088144F6541048818B815D
:1038E00042F29860C88142F2AA40088242F65060D3
:1038F000488240F6980088824FF4FA60C8823D48BA
:10390000903815E00B8145F6B220488145F6C40099
:10391000888143F6E410C88143F2F67008824B8236
:103920004FF44860888240F61C40C88231486038B5
:1039300088610A77F0BD0B814C8146F6340088819E
:1039400044F64230C88144F26670088245F2FA209B
:10395000488241F20400888240F63C70C8822548C3
:103960003038E5E70D814FF4F740488147F6921073
:103970008881CE810B824F8241F25C20888241F2A5
:103980003010C8821B483030D2E700E015E00C81CF
:10399000A1F80AC048F603108881CF8146F27C0066
:1039A000088247F2C830488241F27C50888241F256
:1039B0005040C8820F486030BAE748F23930088179
:1039C0004AF2192048814AF22B00888147F2A470FC
:1039D000C88147F2B6500882A1F812C041F6902083
:1039E000888241F63800C88202489030A0E7000083
:1039F00068040020A2C4000830B54FF4807425028A
:103A00000822102340292ED010DC072925D007DCFE
:103A1000042924D005291DD0062900D1846030BD99
:103A200008291ED02029FAD1026130BDB1F5806F7E
:103A30001FD008DCA14218D0B1F5007FF5D1816913
:103A400021F0020118E0A94218D0B1F5003FECD1F5
:103A5000436030BD0121816030BD856030BDC260F2
:103A600030BDC36030BD036130BD816921F001010B
:103A700002E0816921F00401816130BD426030BD06
:103A8000094910B588424FF0010101D14C0601E00F
:103A90004FF08064204606F02DFB2046BDE8104024
:103AA000002106F027BB000000640040202209B17D
:103AB00002617047C2607047F0B5827A2F4D0121D4
:103AC00091402A6842F001022A602C4E1C3632686E
:103AD0008A433260294A047B294B0C32A4B914680A
:103AE0008C4314604488C78844EA0744877A03EB10
:103AF000C707C7F840460488878844EA0744877A9E
:103B000003EBC707C7F84446047B012C12D11468A5
:103B10000C431460847A026803EBC4044FEA324217
:103B2000C4F84026847A426803EBC4034FEA324269
:103B3000C3F84426114AC37A121D002B136806D01D
:103B40000B4313600D4A0389143213B104E08B4315
:103B5000F7E713688B4313600389012B02D11368C5
:103B60000B431360407B012802D13068084330606A
:103B7000286820F001002860F0BD000000660040C9
:103B800000600040002A426901D00A4300E08A43F5
:103B90004261704710B50368002223F002030360FE
:103BA000036843F0010303604FF6FF7300E0521C0B
:103BB0004468E40701D19A42F9D14268D2073ED065
:103BC0008A79012A02683CD022F080020260CA7918
:103BD000012A026838D022F0400202600A7A012AE3
:103BE000026834D022F0200202604A7A012A026878
:103BF00030D022F0100202608A7A012A02682CD0AA
:103C000022F008020260CA7A012A026828D022F053
:103C1000040202608A78CC78920742EA04620C7946
:103C200042EA04424C79098842EA0452491E0A4396
:103C3000C261016821F001010160002114E000204F
:103C400010BD42F08002C1E742F04002C5E742F0F9
:103C50002002C9E742F01002CDE742F00802D1E7A6
:103C600042F00402D5E7491C4268D20701D09942CC
:103C7000F9D14068C007E2D1012010BD10B400EBBB
:103C80000113D3F8B04114F004041472D3F8B04116
:103C900030D0E4085460D3F8B04104F00204547208
:103CA000D3F8B44104F00F049472D3F8B441240A59
:103CB000D474D3F8B841D472D3F8B841240A147339
:103CC000D3F8B841240C5473D3F8B841240E94733C
:103CD000D3F8BC41D473D3F8BC41240A1474D3F88C
:103CE000BC41240C5474D3F8BC311B0E937410BC2B
:103CF000FFF7DCBE640D1460CDE730B5024600204E
:103D000093685B0108D49068000101D5012003E0AD
:103D10009068C00037D5022002EB0012D2F8803143
:103D200003F00103C2F880310B7A73B3D2F88041FB
:103D30004D681C434B7A43EAC5031C43C2F88041DB
:103D40008B7A03F00F038B72D2F8843123F00F03C8
:103D5000C2F88431D2F884318C7A2343C2F884319A
:103D6000CB7ACC6843EA0423C2F88831CB7B09695B
:103D700043EA0121C2F88C11D2F8801141F001010F
:103D8000C2F8801130BD042030BDD2F880314C7AA9
:103D900023430C8843EA4453C2F88031D0E7000043
:103DA0002DE9F0411B4F1C491C4C7878B1FBF0F019
:103DB000B4F9161048430014E08108BF4FF6FF70B5
:103DC0001DD007F068FE06460D46B7F9060007F05D
:103DD00062FE6FF0060208F052FA0022104B07F064
:103DE00085FE32462B4607F0A1FC00220D4B07F062
:103DF0007DFE00220C4B07F099FC07F01FFE20818E
:103E0000E18880B288422CBF401A00206081BDE862
:103E1000F08100005004002000A60E0020040020C5
:103E2000004CED4000004940000059401248818A92
:103E3000322998BF002206D94289B2F5007F88BF97
:103E40004FF4007200D942810C4A927892003C29CA
:103E500098BF101D0CD9642998BF02F1080007D93A
:103E60004089202828BF202002D2082898BF082097
:103E700003490881704700002004002094040020BA
:103E800074030020F8B5624C4FF448734FF47A7E07
:103E900062685E495A435F4BB2FBFEF21B89888B16
:103EA00003EBC306898A06EB031602EBC6026260C7
:103EB000B2FBFEF20D4692B203B90022814213D941
:103EC000238883420BD9181A80B28B420AD9591B16
:103ED000814200DA88B228B1834201D3181A2080C7
:103EE000218802E00120F7E721804B484C4C837A7F
:103EF0004A4880F89730A6880A23B6FBF3F7B6FB4A
:103F0000F3F680F89870474F360A3F7806EB87063D
:103F1000677F06EBC70606EB811680F89960890873
:103F200080F89A104049414F0E7A80F89B6080F8E3
:103F30009C20002680F89D6080F89E6080F89F603D
:103F400080F8A060A0F89520E288A0F84A20FA88BE
:103F50006424B2FBF4FCB2FBF4F2A0F848C07F8802
:103F6000A0F8D070A0F8BC20314AA0F8C0509588C5
:103F7000B5FBF4F4240694FBF3F3C0F8C83092794F
:103F8000120692FBFEF2C0F8CC202A4A90F8A2302A
:103F900093700246B0F8B44092F8A1200CB9DB0748
:103FA00001D0092305E012F00F0304D0FF2404EB35
:103FB00043034B7000E04E7054090B78120964F310
:103FC000451362F341030B70C3F34011A0F8C61010
:103FD000808D202818D11848017811B10078032865
:103FE00012D140F20110ADF80000012269461348D9
:103FF00006F054F912480168124A01F4E0611143D5
:104000000160BFF34F8FFEE7F8BD000020040020E1
:104010003800002094030020880400209002002033
:10402000680400202200002094040020FA030020ED
:10403000C803002074030020690200200028000843
:104040000CED00E00400FA05174810B5026941685C
:104050000A231144B1FBF3F414494C63046822446D
:10406000B2FBF3F28A6382684A64C28ACA63104C64
:10407000008B0864E089A8B1B0F5807F12D00220DF
:10408000088091F8A50080070BD1E078C00608D41D
:1040900003F022F907490120C870E07840F01000D1
:1040A000E07010BD0020EBE7A0040020900200208B
:1040B000740300202800002010B5022000F08EF8C4
:1040C000002802D001490720486010BD00000240CE
:1040D000C10002D502490860704702494860704734
:1040E00004040240000002400029016802D041F0AF
:1040F000010101E021F0010101607047016821F038
:10410000010101600021016041608160C1603149AD
:10411000304A0839904203D1486840F00F0006E069
:104120002C4A1432904204D1486840F0F0004860B4
:104130007047284A2832904203D1486840F47060A2
:10414000F5E7244A3C32904203D1486840F470407D
:10415000EDE7204A5032904203D1486840F4702085
:10416000E5E71C4A6432904203D1486840F470008D
:10417000DDE7184A7832904203D1486840F0706019
:10418000D5E7154A111F904203D1086840F00F008F
:1041900006E0114A1432904204D1086840F0F00061
:1041A000086070470C4A2832904203D1086840F4F6
:1041B0007060F5E7084A3C32904203D1086840F449
:1041C0007040EDE7044A50329042EAD1086840F46A
:1041D0007020E5E708000240080402400246002083
:1041E000D10001D5034900E003490968114200D01C
:1041F00001207047000402400000024030B5026810
:1042000047F6F0739A430C6A8B682343D1E904455F
:104210002C4323438C692343CC6923434C6A2343B7
:104220008C6A234313430360CA6842600A68826051
:104230004968C16030BD704730B5044600234FF473
:104240007A7504E0284600F005F85B1C9BB2A34297
:10425000F8D330BD002206E00021491C89B20F29A5
:10426000FBD3521C92B28242F6D370472DE9F04143
:1042700002F086FD8C4C012100256076227E002A0A
:104280002DD0A37E00F0040703F00408DFF81CC261
:104290000222874E47455BD1BCF90070B7F57A7FA3
:1042A00056DDB4F84E70B7F57A6F28BF22740BD282
:1042B000B7F5FA6F05D994F81080B8F1000F08BF70
:1042C00021747F1CA4F84E70E77E002F1FBFA77CCF
:1042D000002F677C042F0ED0277F2FB10BE0A07634
:1042E000E5762176BDE8F081677F002F1FBFA77FAD
:1042F000002F0427677400F0020803F00207B84596
:1043000067D1BCF90070B7F57A7F62DDB4F8507000
:10431000B7F57A6F28BF22740BD2B7F5FA6F05D9BB
:1043200094F81080B8F1000F08BF21747F1CA4F826
:104330005070E77E002F1CBFA77C002F19D0677C30
:10434000022F1CBF277F002F13D0677F6FB110E0B3
:10435000B6F91670322FC8BF2574A4F84E502177D5
:10436000677C042F08BF6574C5E7A77F002F18BFBF
:104370006274C707B7EBC37F38D1BCF90030B3F51F
:104380007A7F33DDB4F85230B3F57A6F28BF2274E8
:1043900009D2B3F5FA6F03D9227C002A08BF217431
:1043A0005A1CA4F85220E27E002A1CBFA27C002ADC
:1043B0000BD0627C012A1FBF227F002A627F002A65
:1043C00003D0A27F002A08BF6174A076E07EF8B90E
:1043D00019E0B6F91670322FC8BF2574A4F85050F2
:1043E0006177677C022F08BF6574C2E7B6F91620B3
:1043F000322AC8BF2574A4F85250A177617C0129E4
:1044000008BF6574E1E7A07C10B125776577A577D3
:10441000A07C284FE076387801281CBFB6F916003A
:104420000A28A8BFBDE8F08102F024FCA4F84E5091
:10443000A4F85050A4F85250B18A322988BFBDE880
:10444000F0811D494988B1F5BA5F88BFBDE8F081A8
:104450001A490989002918BFBDE8F0811849CA78AE
:1044600012F0010F06BF0A7C002ABDE8F0813A78FD
:10447000032A1EBF3A78002ABDE8F081A27C002AF8
:104480001ABFE27E002ABDE8F081002814BF072889
:10449000BDE8F081A574C88930F00400C88108BF68
:1044A0003D70BDE8F0810000980100206A02002004
:1044B0002004002069020020C8030020940300208B
:1044C00074030020154810B50121A0F8A91005219A
:1044D00080F8AB102D2141864FF4A071018640F683
:1044E0005801C185002180F8A11018220CA10A30C2
:1044F000FEF701FF0948152210A15330FEF7FBFE1D
:10450000064815220DA16830FEF7F5FE0348182273
:10451000BDE8104002A17D30FEF7EDBE9002002004
:10452000556E6B6E6F776E2020202020202020207B
:10453000202020202020202000000000556E6B6EDF
:104540006F776E2020202020202020202020202077
:1045500020000000194810B519494288A1F8A92087
:10456000027981F8AB20C2884A8602890A8642898C
:10457000CA85027B81F8A120807B81F8A2000F49C7
:104580000F48182210310A30FEF7B5FE0B490C48CF
:10459000152228315330FEF7AEFE0849084815228F
:1045A0003E316830FEF7A7FE044905481822543111
:1045B000BDE810407D30FEF79EBE00004410002094
:1045C0009002002070B5234D062000242880224848
:1045D0001822B0F8A910698090F8AB10A980418E1C
:1045E000E980018E2981C18D698190F8A110A9818E
:1045F00090F8A2001849E8810A3105F11000FEF791
:104600007AFE15491522533105F12800FEF773FE95
:1046100011491522683105F13E00FEF76CFE0E4986
:1046200018227D3105F15400FEF765FE002035F8B3
:104630001010401C214480B28CB26328F7D3A5F837
:10464000C64064220349054805F028FE04490020BD
:10465000C87070BD441000209002002000EC0008DB
:104660002800002070B5194C207801282CD100209A
:1046700006F054F800F04CF9154D284600F0ECF81F
:1046800004281BD113480188284600F023F912485A
:104690000188A81C00F01EF910480188281D00F0B0
:1046A00019F90F48807B000602D445F2757101E0CC
:1046B0004FF6FF710648801D00F00CF900202070B5
:1046C000BDE8704000F0FEB870BD00008801002019
:1046D00000F00008900100209201002094010020C9
:1046E000740300202DE9F041134E3078002821D0CA
:1046F00072B6002006F012F800F00AF90F4D2846B5
:1047000000F0AAF80027042810D10D4CDFF83480FF
:104710006780608838F8101005EB400000F0DAF888
:104720006088401C80B260800728F2D3377000F0A8
:10473000C9F862B6BDE8F081A401002000F40008C9
:104740004A000020AC1100202DE9F041DFF86C8018
:1047500098F8000000282ED072B6002005F0DEFF89
:1047600000F0D6F8164F384600F076F800260428F8
:104770001CD11448144D164C0068010C2980688027
:1047800012480078A880EE802E816889401C6881DC
:10479000A680A08835F8101007EB400000F09AF8CA
:1047A000A088401C80B2A0800628F2D388F8006060
:1047B00000F088F862B6BDE8F0810000A301002097
:1047C00000F8000808020020BA110020A50100200E
:1047D0004A00002030B517490888174A10804888D9
:1047E000164A10808888164A1080C888154A002307
:1047F000164C1080144A1380108801EB4005B5F860
:10480000005424F81050401C80B210800728F3D3C5
:104810000F4C1380108801EB4005B5F8005824F8C0
:104820001050401C80B210800628F3D30948037052
:1048300030BD000000F0000890010020920100202F
:1048400094010020960100204A000020AC110020B5
:10485000BA1100208801002070B50E4E0546304682
:1048600000F062F8042813D10B4C206940F00200DC
:1048700020616561206940F040002061304600F011
:1048800053F8052804D0216941F6FD7211402161D9
:1048900070BD0000FFFF0F00002002400849042007
:1048A000CA68D20701D001207047CA68520701D5F3
:1048B00002207047C968C906FBD503207047000075
:1048C000002002400248016941F080010161704707
:1048D00000200240F0B506464FF6FF770D463846F9
:1048E00000F022F804280FD1084C206940F00100A4
:1048F00020613580384600F017F8052804D021697A
:1049000041F6FE7211402161F0BD0000002002401E
:1049100003480249416003494160704723016745EC
:1049200000200240AB89EFCD00B50346FFF7B6FF8C
:1049300002E0FFF7B3FF5B1E012803D0002B00D17C
:10494000052000BD002BF4D1FAE700002DE9F0416D
:1049500000244FF4C878254642465A495A4805F083
:1049600091FC58484FF4C77630F81410641C294461
:10497000A4B28DB2B442F7D901880124534F0C2957
:1049800003D1B0F81E03A84210D0FFF7C1FF504872
:10499000FFF762FF4F48FFF75FFF4F48FFF75CFFED
:1049A000FFF790FF05F0FEF83C7001E005F0A8F974
:1049B0000025424649494A4805F064FC4749002021
:1049C00031F81020401C2A4480B295B2B042F7D989
:1049D00008880C2803D1B1F81E03A84203D000F0C8
:1049E00009FB7C700BE014223E48891CFEF783FC17
:1049F0003A493C48142216311430FEF77CFC00255D
:104A000014223949394805F03DFC3749002031F876
:104A10001020401C2A4480B295B21328F7D30A888C
:104A200033480026092A02D1CA8CAA4205D0466022
:104A3000066006838660BC7012E08A884B8802EBB1
:104A4000034242600A89CB8802EB034202608A89F2
:104A50004B8902EB03428260C989018302F03CFC6E
:104A60002149002564222831224805F00BFC1E490B
:104A70000020283131F81020401C2A4480B295B221
:104A80006328F7D30888062803D1B1F8C600A842E6
:104A900003D0FFF717FDFC7001E0FFF75BFD16493F
:104AA00040F27143B1F90620487842435A438A6084
:104AB00000044FF47A52B0FBF2F0C8600F48068051
:104AC000BDE8F081DC09002000E00008280000209B
:104AD00000F0000800F4000800F80008FC0C0020BA
:104AE00000E40008BC0400201C10002000E80008BE
:104AF000A004002000EC0008500400201400002056
:104B00001B4810B5017811B1007803282FD119483E
:104B1000C07848B118480168184A01F4E0611143AF
:104B20000160BFF34F8FFEE71548017819B1BDE86A
:104B3000104005F09DB9417819B1BDE8104000F072
:104B40009FBA817819B1BDE8104004F01BBFC0784E
:104B500018B1BDE81040FFF735BD0A4800780028BD
:104B600005D0FFF7BFFDBDE81040FFF7EDBD10BD5C
:104B700069020020940400200CED00E00400FA0516
:104B8000280000209D010020F0B5CC78002204F020
:104B90000F03E40601D58C7823430C784FF00F0CFB
:104BA00014F0FF0F4FF0010E1BD005680E880EFAAF
:104BB00002F42640A64210D196000CFA06F725EA28
:104BC000070703FA06F5CE783D43282E02D0482E7B
:104BD00002D002E0446100E00461521C082AE5D3DF
:104BE00005600A88FF2A1CD94468002202F10806E1
:104BF0000EFA06F50E882E40AE420ED196000CFA43
:104C000006F7BC4303FA06F7CE783C43282E00D1C2
:104C10004561CE78482E00D10561521C082AE5D3A3
:104C20004460F0BD41F480328261816182618169BA
:104C300080697047F0B5144C002801DAE36900E0A0
:104C40006368450D2E0185B2C0F30157B540C0F32E
:104C50000342032F05D0C6020AD503269640B3436C
:104C600007E023F07062636823F07063636002E022
:104C7000AB4343F0706201B12A43002801DAE261DC
:104C8000F0BD6260F0BD000000000140024600205F
:104C900092680A4200D0012070474FF6FF710180F0
:104CA000022181700421C17070470AB1016170470F
:104CB000416170472DE9F003254F264DA7F16006AD
:104CC000D7F80090288CC9F34E0195F80080091A96
:104CD000002226F81810B6F90010B6F902C03046C6
:104CE0005FF0070330F9044F6144B0F902C0224479
:104CF0005B1EF7D18818B6F91E10084408F10101AF
:104D0000C9B22970102924BF00212970B968124B3B
:104D10000A0DDFF848C09A827A680830530CACF864
:104D20000030C1F34E030E4900118B80BB89C3F3E1
:104D30004E03CB800B4908800B49C2F34E0008801C
:104D40000A494FEA59400880BDE8F0037047000067
:104D50006C110020D000002074030020FA03002012
:104D60001A0000208804002068040020C8030020E6
:104D70002DE9F0414FF00108264F274E4446787D3B
:104D8000002500284FF0400130462FD0FFF77EFF6E
:104D900045EA400580213046FFF778FF05434FF490
:104DA00080713046FFF772FF45EA8000C1B20029EA
:104DB0001CBF0729BDE8F08104F10100C4B2042C36
:104DC000DDD30024204605F0A9FC1448C470817C82
:104DD000002908BF80F812801148C18941F0040100
:104DE000C181104903200870BDE8F081FFF74EFF34
:104DF00045EA400580213046FFF748FF45EA80003C
:104E0000C5B24FF480713046FFF740FF40EA05011C
:104E1000CDE7000050040020000C01409801002064
:104E2000740300206902002010B5234B2349B3F915
:104E30002E00B1F90620904200DAC880B3F9302084
:104E4000B1F906108A420EDB501A80B231B1202827
:104E500000D92020824203DD101A02E08020F9E709
:104E60000020188610BD1648B0F90000824200DA12
:104E70001886144A948A502C02D9B0F5FA6F04DAD5
:104E8000114880788000001D07E05089202801D952
:104E9000202002E0082800D20820B3F930404FF467
:104EA000C872944200DA1A86B3F93020104488425E
:104EB000D7DB198610BD0000C80300205E0000206B
:104EC0006C0200202004002094040020F0B52C4E39
:104ED0002D4A2C4BB6F8B210108800244FF4BA5566
:104EE00044F6903739B9B6F8B41021B19988A9427F
:104EF00004D29D8004E09C80508006E0B94203D239
:104F0000998801F57A71998051805188B94200D30E
:104F10005780642141434FF4F877B1FBF7F191805A
:104F20006421A0F5BA50484343F2504190FBF1F0A0
:104F3000C0B29071642801D964209071B6F8C400A1
:104F4000124EC0B95088A84215D99D789DB9957B5D
:104F50008DB10F4DED78ED060DD4B2F92E20A0F5F0
:104F6000BA505043B0FBF1F0D8807078002801D0DF
:104F700074703470F0BDDC8001207070F0BD0000F2
:104F8000900200205E000020C803002022000020C4
:104F900074030020FEE710B545F2555000F024F8E8
:104FA000022000F015F8BDE810407F2000F016B890
:104FB00002494CF6CC4008607047000000300040C9
:104FC00002494AF6AA2008607047000000300040FD
:104FD0000149486070470000003000400149886086
:104FE0007047000000300040014908607047000031
:104FF0000030004070B5142214A11A48FEF77BF966
:105000001848142218A11438FEF775F915483425EC
:105010001438352405704470312282703021C170FB
:105020003223037141718171C27101723926467256
:1050300033268672C3720173457338218173C2733C
:105040000474437437228274C17470BD4D312D31A4
:1050500042452D31202020202020202020202020EB
:1050600000000000D004002020202020202020204C
:1050700020202020202020202020202000000000B0
:1050800070B5134D0C210024298014221149A81C4D
:10509000FEF731F90F491422143105F11600FEF71D
:1050A0002AF900214FF4C77035F81120491C224419
:1050B00089B294B28142F7D9A5F81E434FF4C87261
:1050C0000349054805F0EAF804490020487070BD1E
:1050D000FC0C0020BC04002000E400082800002094
:1050E00010B5002402F070F8641CA4B2642CF9D34B
:1050F0000448417B012903D1C18941F48051C18118
:1051000010BD0000740300200C4910B5C88840F69B
:10511000AB54431E0A4AA34208D2098801EB81011D
:105120004900B1FBF0F01169084410611169106881
:1051300008440A21B0FBF1F0D06010BD200400202B
:10514000A004002070B45B485B4AB0F90C300382C5
:10515000B0F90E1003EB410151430C14448257493E
:10516000564A0988128801F50041890911F44075F1
:1051700002F500425249C2F38712C2F1FF0C7CD003
:10518000B5F5807F7AD0B5F5007F03D0B5F5407FC7
:1051900006D00DE031F81220028131F81C1006E033
:1051A00031F81CC0A0F808C031F8121077E0418136
:1051B000B0F90A20B0F9085003FB02F104FB151105
:1051C0006B43CE1304FB02323E4990F801C0D31367
:1051D00001F1200221F81C6022F81C30B1F90030E6
:1051E000B1F90250B2F900401D44B2F90230234433
:1051F000B1F90440B1F906102C44B2F9045021442D
:10520000B2F90620891C2B4489101A44C183911CD1
:105210000CF1010241F38F01D2B281824270042A63
:1052200004BF002242704A422749B1F9003003FB13
:1052300002F4B1F904305A434B694FEAE37C9B18FE
:105240004CEBE272D1F810C04FEAEC75BCEB0306F0
:10525000954109DBD1F80CC04FEAEC75B3EB0C06B5
:10526000AA41A8BF4B6101DAC1F814C04A69B1F97B
:105270000A302244D213934201E00AE011E0AABFAF
:10528000B1F908101A469142C8BF0A46428370BC61
:10529000704731F812205242028131F81C10494205
:1052A00085E731F81CC0CCF1000CA0F808C031F83B
:1052B00012107CE7D0000020326CFFFFF8010020C4
:1052C00064C500082C110020FC0400202DE9F041E9
:1052D000324C012100256078314ECF0370B1012896
:1052E00040D0022808D1A078401CC0B2A07003288A
:1052F00002D3A570E5706570BDE8F081294800789B
:10530000012811D0284A0020D28901FA00F31A425C
:105310000ED0A5702571401CE070617000223946E6
:105320003046FFF7C2FC07E000223946304615E060
:10533000401CC0B21028E8D3E0780028DCD1A07867
:10534000401CC0B2A0700228D6D3A570B168304608
:10535000090401D5002200E001223946BDE8F041F0
:10536000FFF7A3BC2079401C2071B068000401D570
:10537000002200E0012239463046FFF796FCE07833
:1053800021794000801C8842B6D2A570002239469F
:105390003046FFF78AFC02206070ADE788000020ED
:1053A0000010014069020020740300203D49B1F95A
:1053B0000230B1F90420934208BF70473A4890F890
:1053C00001C0BCF1010F18BF704730B4DFF8DCC07A
:1053D000BCF81440782C32D8DFF8D4C09CF80140D7
:1053E00014F0040F1DBF9CF804C0BCF1000F4FF077
:1053F000040C4FF0080CC48804F10104A4B2C4806A
:1054000064459CBF30BC70474FF0000CA0F806C04C
:1054100003F1200C23489445B0F900001DDA254C17
:105420002488242C19D20FFA8CF24A809042DCBFD7
:1054300030BC7047B0F5E06F1FDD30BC7047BCF882
:105440000A50DFF874C01D4C0A2D9CF801C014F8F6
:105450000CC088BF4FEA5C0CCDE703F1100C9445FB
:105460000EDA0FFA8CF24A809042DCBF30BC7047F3
:10547000B0F5E06FC4BF30BC7047488030BC7047A7
:1054800002F1200C6345DEBF4A8030BC7047A3F1B7
:10549000200212B24A808242C8BFEF28EDDC30BC45
:1054A00070470000880400206802002020040020CB
:1054B00074030020BE010020940400206CCC00087E
:1054C00008480078002808BF70470748007B00287C
:1054D00018BF7047002005494861054948610549E2
:1054E000088070479D01002074030020FC04002008
:1054F000E4040020EA000020094910B500204861BA
:10550000084948610849088000F0A0FD0748C08AA2
:10551000002818BF10BDBDE8104000F089BD000094
:10552000FC040020E4040020EA0000202004002005
:1055300070B5324C207800281CBF2078032807D192
:105540002F494FF0EF0048804FF0000005F0E6F8DB
:10555000217800222B48012948D02B49B1F9163077
:105560000A2B43DA898A322940D228494988B1F581
:10557000BA5F3BD226490989002901BFC17811F0E1
:10558000010F017C002931D1C18911F0080F04D02D
:10559000204B1A7021F00801C1818BB21E4913F013
:1055A000400F08D0B1F800C00D89AC4503D94A7747
:1055B00023F04003C3819BB213F4006F09D0DFF8DE
:1055C0005CC0BCF80AC0BCF1040F3CBF23F400630C
:1055D000C3819BB213F0200F08D0B1F800C08D89B1
:1055E000654503D98A7723F02001C18121780329F9
:1055F00002BFC0890028227070BD0000690200202F
:10560000880400207403002020040020C803002028
:1056100094030020A80100206804002094040020C6
:105620002DE9F04FDFF838C48EB00022BCF90060DD
:10563000BCF902300193F31A114610460D9348BF8E
:105640005B42DFF81CC4019CBCF904C0B4EB0C0C39
:10565000CDF828C04CBFA3EB0C036344102BB4BFA0
:105660001023B3F5006FC8BF4FF40063FD4CB4F9CD
:105670000070B4F902C0CDF800C0B7EB0C0CCDF847
:1056800030C048BFCCF1000CF64C009DB4F904408A
:105690002C1B09944CBFACEB040CA444BCF1100FC0
:1056A000B4BF4FF0100CBCF5006FC8BF4FF4006CD6
:1056B000DFF8B483B8F90050B8F90290B5EB0904EB
:1056C0000B9448BF6442DFF8A083B8F90480B9EBBB
:1056D0000808CDF820804CBFA4EB08044444102CEB
:1056E000B4BF1024B4F5006FC8BF4FF40064DFF8F6
:1056F0007C8398F803A0BAF1000F14BF4FF0010BA0
:105700004FF0000B88F804B0DFF8608398F807B01A
:10571000B8F826E0CDF81CE0B8F824E0CDF818E0A1
:1057200008F13A0EBBF1070FBEF900E00EEB4E0E8A
:10573000CDF814E0B8F82280CDF81080DFF820838F
:10574000B8F9008008EB4808CDF80C80DFF8188322
:10575000B8F9008008EB4808CDF80880DFF810831E
:1057600080F01C83DFE80BF0FE0483FDFCFBFA00F5
:10577000C04801680798BD4A401A10F5804FB4BF71
:105780004046B0F5804FC8BF4FF48040411BA14256
:10579000C8BF281904DCC4F1000B8B45C8BF281B07
:1057A0001063BAF1000F1DD0B3490C680699091BAC
:1057B000CC1BB4F5805F02DC14F5805F01DA0024B5
:1057C000147111F5804FB4BF4146B1F5804FC8BF89
:1057D0004FF48041CA1B62452ADCCCF10004A2428E
:1057E0002FDA2CE0411B48BF49420C9A002A099A43
:1057F00009D4002A58BF39440ED5059A0A440099A5
:10580000511A491008E0002A48BF791A04D4059AB1
:10581000521A0099511A491011F5804FB4BF4146F0
:10582000B1F5804FC8BF4FF48041CA1B624502DD0D
:1058300007EB0C0105E0CCF10004A24201DAA7EB72
:105840000C010A18524212F5804FB4BF4246B2F51D
:10585000804FC8BF4FF48042A2EB060C9C4500F37A
:1058600097825C42A44580F2998200F096BA814802
:10587000026807987D49801A10F5804FB4BF4046F2
:10588000B0F5804FC8BF4FF48040421BA242C8BF52
:10589000281904DCC4F1000B9345C8BF281B08631A
:1058A000BAF1000F1CD0744A1468049A121B941B9E
:1058B000B4F5805F02DC14F5805F01DA00240C711E
:1058C00012F5804FB4BF4246B2F5804FC8BF4FF4C7
:1058D0008042911B994229DC5C42A1422CDA2AE0E9
:1058E000411B48BF49420D9A002A0A9A09D4002A4E
:1058F00058BF72180ED5039A0A440199511A4A10DA
:1059000008E0002A48BF721A04D4039A521A019977
:10591000511A4A1012F5804FB4BF4246B2F5804F7B
:10592000C8BF4FF48042911B994201DDF21803E099
:105930005C42A14200DAF21A1118494211F5804F77
:10594000B4BF4146B1F5804FC8BF4FF48041CB1B77
:1059500063457DDCCCF10004A34204E099E113E14E
:1059600095E003E012E280F219828CE0424802687E
:1059700004983E49821A12F5804FB4BF4246B2F5F0
:10598000804FC8BF4FF48042901B9842C8BFF218A6
:1059900004DCC3F1000B8345C8BFF21A0A63BAF1F5
:1059A000000F1CD0334803680798C01A431BB3F597
:1059B000805F02DC13F5805F01DA00230B7110F5C4
:1059C000804FB4BF4046B0F5804FC8BF4FF4804011
:1059D000411BA14229DC634299422CDA2AE0901B48
:1059E00048BF40420B990029089909D4002958BFA3
:1059F00028440ED502990844A0EB0900401008E0A5
:105A0000002948BF281A04D40299081AA0EB0900FB
:105A1000401010F5804FB4BF4046B0F5804FC8BF6E
:105A20004FF48040411BA14201DD281903E063428D
:105A3000994200DA281B1118494211F5804FB4BF72
:105A40004146B1F5804FC8BF4FF48041CB1B00E009
:105A500001E0634512DD07EB0C0100F09FB9000087
:105A6000040100200A01002010010020D0000020C5
:105A700000C0FFFF3C2801403C240140CCF1000461
:105A8000A34280F28B81A7EB0C0100F087B9F748A5
:105A900002680499F6488A1A12F5804FB4BF42464C
:105AA000B2F5804FC8BF4FF48042911B9942C8BFE6
:105AB000F21804DCC3F1000B8B45C8BFF21A026375
:105AC000BAF1000F1DD0EB490B680699C91ACB1B20
:105AD000B3F5805F02DC13F5805F01DA0023037108
:105AE00011F5804FB4BF4146B1F5804FC8BF4FF4A8
:105AF0008041C81B60452ADCCCF1000398422FDAB4
:105B00002CE0901B48BF40420C990029099909D408
:105B1000002958BF39180ED5059901440098081A74
:105B2000411008E0002948BF391A04D40599091A20
:105B30000098081A411011F5804FB4BF4146B1F5E5
:105B4000804FC8BF4FF48041C81B604502DD07EBA2
:105B50000C0105E0CCF10003984201DAA7EB0C013F
:105B60005018404210F5804FB4BF4046B0F5804F0A
:105B7000C8BF4FF48040431BA3426EDCC4F1000C4D
:105B8000634580F20B8182E0BA4802680699B84802
:105B9000891A11F5804FB4BF4146B1F5804FC8BF97
:105BA0004FF48041CA1B6245C8BF07EB0C0105DCFE
:105BB000CCF1000B9345C8BFA7EB0C010163BAF110
:105BC000000F22D0A94AD2F800C0049AA2EB0C021E
:105BD000A2EB060CBCF5805F02DC1CF5805F03DAEB
:105BE0004FF0000C80F804C012F5804FB4BF42465D
:105BF000B2F5804FC8BF4FF48042901B98422ADC18
:105C0000C3F1000C60452EDA2CE0C81B48BF4042AF
:105C10000D9A002A0A9A09D4002A58BF32180ED5C4
:105C2000039A02440198101A421008E0002A48BF63
:105C3000321A04D4039A121A0198101A421012F55B
:105C4000804FB4BF4246B2F5804FC8BF4FF4804288
:105C5000901B984202DDF21805E012E0C3F1000C3F
:105C6000604500DAF21A5018404210F5804FB4BF78
:105C70004046B0F5804FC8BF4FF48040431BA3425D
:105C800001DD28198AE0C4F1000C63457EDA281B87
:105C900084E0764801680698754A411A11F5804FEC
:105CA000B4BF4146B1F5804FC8BF4FF48041C81B17
:105CB0006045C8BF07EB0C0105DCCCF1000B834548
:105CC000C8BFA7EB0C011163BAF1000F22D06948DD
:105CD000D0F800C00798A0EB0C00A0EB050CBCF5B9
:105CE000805F02DC1CF5805F03DA4FF0000C82F865
:105CF00004C010F5804FB4BF4046B0F5804FC8BF18
:105D00004FF48040421BA2422ADCC4F1000C6245E1
:105D10002DDA2BE0C81B48BF40420B9A002A089A94
:105D200009D4002A58BF28440ED5029A1044A0EB8B
:105D30000900401008E0002A48BF281A04D4029A3B
:105D4000101AA0EB0900401010F5804FB4BF404678
:105D5000B0F5804FC8BF4FF48040421BA24201DD26
:105D6000281904E0C4F1000C624500DA281B0A1867
:105D7000524212F5804FB4BF4246B2F5804FC8BFC1
:105D80004FF48042A2EB060C9C4500E006E001DDEA
:105D9000F21803E05C42A44500DAF21A364B1B7895
:105DA000012B3ED0354900208B1D888001F10C026B
:105DB00098809080488058805080088018803439BE
:105DC000108008632D48B0F90020343800F13A0102
:105DD0008281B1F90010C181D0F830C0BCF1000F50
:105DE000B8BFCCF1000C264BB3F906309C4513DC50
:105DF000002AB8BF52429A420EDC0029B8BF49427D
:105E0000994209DC1F49B1F900100029B8BF494285
:105E10009942D8BF002100DD012181710EB0BDE89B
:105E2000F08F164BDDF804C0A3F804C003F1060C94
:105E3000009CACF8044003F10C04A4F804905E80CC
:105E4000ACF8027065801A80ACF800102080A3F1D5
:105E50003400016B11F5804FB4BFC0F83080B1F54C
:105E6000804FC4BF4FF480410163ABE73C24014045
:105E7000D00000203C2801406902002004010020DD
:105E800088040020100100202DE9F041604C614D94
:105E9000DFF884816078614F10F0020F4FF0010647
:105EA00008D004F0A9F8B7F93000B5F930108842ED
:105EB0000CDD0AE010F0040F08D005F03BF8B8F94B
:105EC0001000B5F93010884200DD267160784FF07F
:105ED000000610F0010F18D0FEF7A6FF607810F052
:105EE000020F07D0B5F9300078B1B7F93010884209
:105EF0000ADA0AE010F0040F06D0B5F9300020B13C
:105F0000B8F91010884200DB2671227C44484FF417
:105F1000C8734FF47A717AB1B4F90620B2F5C87F2C
:105F2000B4BFE380B2F57A7FC8BFE18046DAE1888A
:105F300001F10201E18041E0627B0AB1E68060E0AC
:105F4000627C012A12D0E17811F0010F39D0B4F946
:105F5000061040F6B832B1F5C87FB4BFE380B1F5A2
:105F60007A7F15DCE188491CE18022E0B4F9062043
:105F7000B2F5C87FB4BFE380B2F57A7F06DCE28871
:105F8000921C12B2E280B2F57A7F36DDE18038E011
:105F9000244BB3F806C00CF1010C1FFA8CFCA3F8DB
:105FA00006C0BCF1080F04D39142DCBF491CE1805C
:105FB000DE80B4F906109142C8BFE280818C018373
:105FC0001BE019490A78002A1CBF4988E18014D1D6
:105FD000164949780029B1D0217951B1617811F081
:105FE000020F0CBFB8F91010B7F93010E180B98872
:105FF00002E0298EE18069890183B4F90610002945
:106000009CDB818A808BBDE8F04104F08DBA0000F2
:1060100074030020C8030020FA030020940300202A
:1060200020040020500000202200002094040020C2
:1060300005480021C18401858170C1708171C185CD
:106040008184C166704700009801002010B500F0FF
:1060500097FE0149C87710BD980100202DE9F04155
:10606000002600F007FE4B4C0025E07794F8202036
:1060700090427ED0A18F638C99429CBF61790029A8
:106080001AD000BF4FF00107277194F900100029C2
:1060900018BF617025704049895C814208BF277034
:1060A0003AD03E49895C81422AD1208D002804BF24
:1060B0006079002821D113E094F9011094F900309F
:1060C000994218BF002BDDD1238D002B08BF012979
:1060D000D8D0E38C002B08BFB1F1FF3FD2D048E00D
:1060E000E08C062809D9B4F8400040F28A218142A8
:1060F00003D96078207001260EE0FF2020700BE0AD
:10610000E178491CC9B2E170032913D02449085C25
:10611000062818BF01260DD094F9000094F901104B
:10612000884203D0F0B1E57300F05CFE2078C8B17E
:1061300096B117E0E570002004F0F0FAA07C00288A
:1061400008BFA7741748C18941F00401C1811649ED
:1061500003200870E0E70CE0E57000F02FF900F094
:106160005FFEA587E07F84F82000002E08BFBDE811
:10617000F0810E4804F068FB0D490988A28C491C87
:1061800000EB02404843E16E0844E066A584BDE8A8
:10619000F081000098010020380200204002002019
:1061A000480200207403002069020020000800401B
:1061B000280800402DE9F04F7A487949D0F868C0A6
:1061C0000646C47BB6F83480B6F84020DFF8D8E144
:1061D0000023F67F00F1B00701252CB18179A1B130
:1061E000424588BF83711EE017F8069040F2DC5BE1
:1061F0003EF819A00AFB0BFADFF8B0B15BF8299062
:10620000BAFBF9F9A0F82C9013E0C18C0F2984BFD8
:10621000C18E914207D9C18D491C89B2C18513290C
:1062200008BF857100E0C3856149B1FBFCF1818540
:106230006146C0F864C0DFF86CC190F80790BCF804
:1062400032C0B9F1000F05D0B0F830904A4588BF90
:10625000C37104E0002C18BF624538BFC57190F8C7
:106260000890B9F1000F03D0624588BF037204E0C3
:10627000002C18BF424538BF057290F80580DFF842
:1062800024C141F25559B8F1000FBCF954C006D1F0
:10629000DFF8208198F80080B8F1010F05D0A0F850
:1062A0005630A0F82AC0837371E0DFF8F8A090F8A8
:1062B0000EB0BAF82A80BAF854A0BBF1000FAAEBCE
:1062C00008080FFA88F839D0C279002A08BF83730A
:1062D000B0F92C30428F93424CDD048F9A1A92FB16
:1062E000F4F292B20C2A88BF0C22DC0004EB4303C8
:1062F0001BB24B45C8BF41F25553B8F1000FBABFAE
:10630000C8F1000424B24446E40004EB6304641CB6
:1063100094FBF3F39BB20C2B88BF0C23934228BF52
:10632000002206D2D21A92B2062A84BF921F51438B
:1063300025D2C2F10602B1FBF2F120E0C18C0129A5
:106340009CBFA0F85630A0F82AC00DD9B95D08EB63
:1063500048035B003EF81110594342F6AB235A4301
:1063600091FBF2F1A0F85610002C1EBFC179002954
:1063700085730CE0104AA2FB01214FEA910140F223
:10638000DC5208FB02F292FBF1F1A0F856100CEB84
:106390000901A0F85410B0F92C00BDE8F08F0000FE
:1063A000B0CA0B0198010020941100207C1100203C
:1063B0000000DC0569020020ABAAAAAA70B56C4CEB
:1063C0000025E17F94F8200001F0040200F00403AE
:1063D0009A420CD0B4F84410B4F842000144A4F836
:1063E0004010A4F84400E087A4F8425022E001F0F5
:1063F000020200F002039A420CD0B4F84810B4F83C
:1064000046000144A4F84010A4F84800E087A4F82E
:1064100046500FE0C907B1EBC07F0BD0B4F84C1069
:10642000B4F84A000144A4F84010A4F84C00E087F6
:10643000A4F84A50A08F40086084802884BF802040
:106440006084E07B012118B9E08C072888BFE173E4
:1064500094F90000002808DDE08C4FF6FF718842B7
:106460004FD2E08C401CE0844BE04ADAA571E58510
:10647000208DFF2802D2208D401C2085607A0128C3
:1064800008BF6572A07A012808BFA572208D172861
:1064900037D9B4F84000B0F5A07F32D2354841F684
:1064A0007052B0F9000090422BDD3148667BD0E994
:1064B00022C3D0F88020D0F88400002E1FBF65735F
:1064C000C4E92A20C4E928C3D4E9260201BF6173C4
:1064D000C4E92820C4E92AC3D4E92402C4E92C026F
:1064E000607A022808BF6572A07A022808BFA572E8
:1064F000E07A30B920484089A0F57F42FE3A18BFC3
:10650000E172E18C1D48022902D204F09DF91CE0E1
:1065100004F09AF91A490988A28C491C00EB024040
:106520004843E16EE27F01441648825C164840F819
:10653000221001684268114482681144C268114403
:106540000269406911440844A066A584E566E08CB0
:10655000FF2898BF70BD2078012806BF607C002806
:1065600070BD00F025FBBDE8704000F08DBD00005F
:10657000980100206C020020BA11002000080040A1
:1065800028080040480200207C11002000B500F0DF
:10659000C1F91C48817871B1418D828D891A09B287
:1065A0004185B0F95A20D317B3EBE17F15D1511AC9
:1065B000002912DD10E0818DB0F856201144428D83
:1065C000114409B24185B0F95820D317B3EBE17FEC
:1065D00003D1891A002900DD428502790021002AB1
:1065E00018BF417107D0417B0029418D08BF494246
:1065F000A0F8601000BD01224271B0F8542042851D
:106600008173F0E7980100202DE9F05FB04844F66F
:10661000E741B04C408ADFF8C4C24143AE486167ED
:1066200041F25556028A130442785343B3FBFCF3FC
:10663000B1FBF3FAC4F87CA0A367B0F906305A4363
:1066400040F271435A438260A548A0F1180E838935
:10665000A0F10C05A3F57F42FF3A2BD04788B0F894
:106660000090A7EB09029642D8BFB2F5804F21DC1B
:10667000B0F804C0ACEB07029642D8BFB2F5804F29
:1066800018DCC388A3EB0C029642D8BFB2F5804F4A
:1066900010DC0289A2EB03084645D8BFB8F5804F4D
:1066A00008DCB0F80A80A8EB020B5E45D8BFBBF54A
:1066B000804F2BDD8B488C4A00881388C2182A80B3
:1066C00042F6AA2203EB020C8444A5F802C045F26C
:1066D000555C9C448444A5F804C047F6FF7C9C4468
:1066E0008444A5F806C0A3F5AA4CACF1550C84442B
:1066F0009B1A1844A5F808C06881AEF10200032374
:10670000428020F8042F5B1EFAD127E0A5F8009004
:106710006F80A5F804C0EB802A81A5F80A80038861
:106720004289A3EB020CAEF800C0B0F802C0ACEB9B
:106730000303AEF802308388A3EB0C0CAEF804C060
:10674000B0F806C0ACEB0303AEF806300089A0EB4E
:106750000C03AEF80830101AAEF80A0063480123A3
:106760000027B0F80AC0ACF57F42FF3A0AD0B4F96E
:10677000622040F6AA2C12EB0C0FA4BF40F6AA2C04
:1067800094457DDAC4F870A067746373206F5A4A29
:10679000B1FBF0F04FF42021B1FBF0F12186544918
:1067A000B1FBF0F161865349B1FBF0F1A1864FF4E2
:1067B0000031B1FBF0F1E18664214143A2FB0121EC
:1067C000CA084FF48031B1FBF0F0B1FBF2F2C01C0B
:1067D00080B24AF6AB2148436287800C2087E7727B
:1067E000277300F0FFFAE766A78440F2CF30608499
:1067F000607B002861D0D4E92001C4E92E01D4E9EE
:106800002201C4E93001D4E9240100BFC4E9320106
:10681000D4E92E01C4E92801D4E93001C4E92A01F0
:10682000D4E93201C4E92C01A4F85670A785A771F8
:1068300023706370A773E77300F0A2FA2F49E07723
:10684000095C35F811103144A4F854106185A4F89E
:106850005810A4F85A10A4F85C10A4F85E1084F83C
:10686000200027480780001F07802648018841F044
:10687000010101802448018841F00301018000E00A
:1068800007E0001D4FF6FE710180491E0180BDE842
:10689000F09F0288B0F802C04CEA02422267DFF89B
:1068A0006CC0A2F51032A2F51F62624524BF184ADF
:1068B000226767740079607368E7D4E92201C4E94C
:1068C0002E01D4E92001C4E93001D4E926019DE775
:1068D00068040020980100205004002000A60E004B
:1068E000AC1100201600002014000020BA11002076
:1068F000AAAA06006DDB0200898888884802002069
:1069000028080040000800400C08004051F80C0026
:10691000400D03002A4B00B5988F40F29E718842CB
:106920003CBF401C9887B3F8422041F2DA608242B3
:106930003ABF521CA3F84220A3F84400B3F8462003
:1069400082423ABF521CA3F84620A3F84800B3F88D
:106950004A2082423ABF521CA3F84A20A3F84C00B6
:106960009A8F8A423CBFB3F84210814207D2B3F8F3
:10697000461081423CBFB3F84A1081420AD300203E
:106980001871D87342F6B451A3F840100D49C8826B
:1069900000F028FA587918B9187A08B1987820B117
:1069A000B3F85A00A3F8580000BD987900281ABF20
:1069B000B3F85E00A3F85800B3F85C00F2D000BD55
:1069C00098010020200400207448C17C012918BFD0
:1069D00070477248407A012818BF70472DE9F04F80
:1069E0004FF0000C6E4E87B0301F63466246614622
:1069F00003244568641EAC44C5692B4450F8085F05
:106A0000294485692A44F4D1601E0CEB010703EB8D
:106A1000020800EB57040025394656F8250000FB14
:106A200008F0001904F0FEF846F82500681CC5B20D
:106A3000062DF1D307EB0800401C470859486E4665
:106A400000F14C0191E80E108DE80E10C06D04901D
:106A5000501801901844029060440390DDE903103F
:106A600008440025CDF8100036F82500394600040A
:106A7000001904F0D7F846F82500681CC5B2052DAA
:106A8000F2D349484949008880B20880009A0244FC
:106A900094B24C80019A024495B28D80029A0244CD
:106AA00096B2CE80039A024497B20F81049A0244B0
:106AB0001FFA82F8A1F80A800C31B1F8009048451D
:106AC00004D9A0EB0902B2F5B67F52DCB1F802C0DE
:106AD000644504D9A4EB0C02B2F5B67F49DCB1F8E9
:106AE00004A0554504D9A5EB0A02B2F5B67F40DCF7
:106AF000B1F806B05E4504D9A6EB0B02B2F5B67F3D
:106B000037DC0B899F4203D9FA1AB2F5B67F30DC25
:106B10004A89904504D9A8EB020EBEF5B67F28DC61
:106B2000484504D2A9EB0000B0F5B67F21DC6445EE
:106B300004D2ACEB0400B0F5B67F1ADC554504D2A4
:106B4000AAEB0500B0F5B67F13DC5E4504D2ABEBD3
:106B50000600B0F5B67F0CDC9F4203D2D81BB0F51F
:106B6000B67F06DC90450BD2A2EB0800B0F5B67FED
:106B700006DD8889A0F57F42FE3A1CBF401C888153
:106B80000848D0E90912C36A8363C0E90C120348BC
:106B90000221417207B0BDE8F08F0000980100208B
:106BA000C81100207C11002014000020A01100203A
:106BB00070B42C48467A01462B4DB1F84030CA7F5C
:106BC00000F1B0044FF0010C00219EB1467A012E75
:106BD00007BFC67C002E70BC704740F23E36B34201
:106BE0009CBF2B78012B1CBF4172C1741BD08175D7
:106BF00070BC7047C174B3F5027F24BF70BC70478E
:106C00002B78012B07BFA25C002A70BC7047174A83
:106C100041F67053B2F900209A42AEBF80F809C025
:106C200070BC7047E3E7A25C114B53F82220540973
:106C3000827D4C3343F822404AB103EB820252F882
:106C4000042CB2EB440F02D941728175C174817D6D
:106C5000491CC9B281750C2908BF80F813C070BCEB
:106C60007047000098010020690200206C0200209B
:106C70007C1100202DE9F047DFF8F890002635461A
:106C800099F81F0089F8150000F07AF80446DFF83B
:106C9000E8803A4F39E000BF98F815004FF0000A3D
:106CA00000284FF04001384636D0FDF7EFFF4AEAA2
:106CB000400A80213846FDF7E9FF40EA0A0A4FF40E
:106CC00080713846FDF7E2FF4AEA8000C0B2A04278
:106CD0001BD0681CC5B2002698F815003446002861
:106CE0004FF0400138462BD0FDF7D0FF44EA400476
:106CF00080213846FDF7CAFF04434FF480713846BF
:106D0000FDF7C4FF44EA8000C4B2701CC6B2032E73
:106D100028D2032D28D2BFE7FDF7B8FF4AEA400A80
:106D200080213846FDF7B2FF4AEA800000F0FF0AF2
:106D30004FF480713846FDF7A9FF40EA0A00C6E724
:106D4000FDF7A4FF44EA400480213846FDF79EFF8A
:106D500044EA8000C4B24FF480713846FDF796FFD4
:106D60000443D2E7032D01D399F815402046BDE82E
:106D7000F08700009801002050040020000C014022
:106D800070B516480024164D407D4FF04001002894
:106D9000284610D0FDF77AFF44EA400480212846B7
:106DA000FDF774FF0443A9152846FDF76FFF44EA79
:106DB0008000C0B270BDFDF769FF44EA4004802145
:106DC0002846FDF763FF44EA8000C4B24FF48071A7
:106DD0002846FDF75BFF204370BD000050040020F3
:106DE000000C01400C4840F2DC52B0F84010514316
:106DF0008166818F4A4309490A604A608A60CA6095
:106E00000A614A610021C18401858170C17081716C
:106E1000C1858184C1667047980100207C110020E3
:106E20002DE9F043624C0025214694F901C094F904
:106E30000020604FC97F41F2555840F29E7004F126
:106E4000B00694453FD0E5842585A573725C37F87C
:106E5000122002EB080304F18002A4F85630515CC2
:106E6000715C37F91120A4F85420B4F92AC0A3EBBF
:106E70000C01514B09B2A1851B78012B18BFA585C8
:106E800006D1002912DD490009B291FBF0F0A0857E
:106E9000B4F85600A4F85400A4F85A00A4F85C0012
:106EA000A4F85E00A4F85650BDE8F083A2EB0C01F4
:106EB00009B2A1850029C6BF91FBF0F0A085A58588
:106EC000A4F85620E4E7DFF8F8903C4AA9F1A003C3
:106ED000BCF1010F9B8F31D0BCF1FF3F18BFBDE863
:106EE000F083A573E573D582E584A4F8565001209C
:106EF000A070705C334A32F81020B2FBF3F2A28526
:106F000019F80110715C37F81110618537F810001D
:106F100000EB080109B2A4F85410228D082A32BFF0
:106F2000A4F85A1000F25550A4F85A00B4F85A00C8
:106F3000A4F85C00A4F85E00BDE8F08340F28A2C5F
:106F400063453CBFB4F84230834214D2B4F84630B3
:106F500083423CBFB4F84A3083420CD2207950B10E
:106F6000B4F840004FF4803303EB5003B3FBF0F070
:106F700000B2102800DA0020D082705C37F81000D0
:106F8000A4F85400FFF716F9A085E07F19F8000077
:106F9000305C37F81000A4F85A0000F6AA21A4F8D3
:106FA0005C104044A4F85E00A5702585BDE8F08320
:106FB00098010020A0110020690200202004002078
:106FC00038020020941100202DE9F0412A4E307D36
:106FD000012806BFB07A0128BDE8F0814FF0000C0F
:106FE000264B644603F12002604602F120014FF077
:106FF000100500BF33F8027B6D1EBC4432F8027BE3
:107000003C4431F8027B3844F4D105094FEA1C11A5
:1070100024094FF4803003F005FE1949498A48439A
:10702000214603F0FFFD45F2F4014843294603F0F1
:10703000F9FD0146706F03F0F5FD316FC1F3501299
:107040008B18891A984203D8884228BFBDE8F0817E
:10705000F17A002918BFBDE8F0810A494989A1F5F4
:107060007F42FE3A08BFBDE8F08130670120F07230
:107070000220B072BDE8F08198010020F8110020D4
:1070800068040020BA1100202DE9F00F4848877AE3
:107090004849DFF828C10346474C0126B1F90020D2
:1070A000B3F84030BCF900C041F6705500217FB103
:1070B000877A012F07BF077D002FBDE8F00F7047CB
:1070C00040F23E37BB429CBF2478012C1AD113E01A
:1070D000B2F5B37F0CDA427A022A09D1B3F5027F06
:1070E00006D22278012A03D1AC45A4BF8672C175AD
:1070F0000175BDE8F00F7047AC45A4BF40F2CD2448
:10710000944205DA8172C1750175BDE8F00F7047D0
:10711000DFF8AC80C27D2B4C08F1200728F8123034
:1071200025881FFA8CF427F8125007F1200C08EB81
:1071300042082CF8124038F8028C07EB420708F19D
:1071400010094FEA591A08EB0A0937F802BCA8EBF4
:107150000A080BF110077F090BEB070AABEB0707D7
:107160001FFA89F91FFA88F81FFA8AFABFB2AAB182
:10717000434528BF99450ED3BD4228BFAA450AD32F
:107180000CEB420204F1800332F8022C934202D34A
:107190008032944202D98172C1750175C17D491C4A
:1071A000C9B2C175102908BF0675BDE8F00F704758
:1071B0009801002088040020690200206C02002051
:1071C000F81100206804002030B51448124B144D0B
:1071D00001785C7B0022491C002C2C68C9B24FEA64
:1071E000845409D0002C05DA0170032901D1027002
:1071F0005A7330BD027030BD002CFBDB01700229D8
:10720000F9D1D97821F00101D97006490A700270CC
:107210000120587330BD0000740300208800002056
:10722000080C014022000020F0B52848264F294DC7
:10723000838AB0F916202648FC894FF00006408862
:10724000E1070AD02E70322B1DD80A2A1BDCB0F5BC
:10725000BA5F18D224F0010020E01B4995F802C063
:107260004978BCF1000F1BD02E70322B08D80A2AA7
:1072700006DCB0F5596F03D345F61032904203D3C4
:10728000C80701D06E70F0BD6878401CC0B268704D
:107290000328F8D16E70AE7024F00200F881F0BDC2
:1072A000A0F55960B0F59B4F0BD9C80709D02878D5
:1072B000401CC0B228700228F1D12E700120A870A5
:1072C000F0BD2E70F0BD00007403002020040020EB
:1072D000C80300205E00002003480069002802D097
:1072E0000249012088707047A00400202800002077
:1072F00010B500F019FDBDE8104001F007B800001E
:107300002DE9F047384E4FF4FA69384CB28A4A45B5
:1073100009D3A079022802D2401CA07103E0F078C2
:1073200040F02000F070F178314F88064FF00108EE
:107330004FF0000514D540F2D940824210D8607950
:10734000052802D2401C60710BE0C80609D4FFF783
:10735000C3FF87F80380F07840F01000F07000E081
:107360006571B069B0B12349898A052912D8A1682D
:10737000C0EB0010491C00EB8000A160B1EBC00F16
:1073800009D3FFF7A9FF87F80380F07840F01000D9
:10739000F07000E0A560F078C00621D5B878F8B9A3
:1073A000F878E8B9002003F0B9F913480570002215
:1073B0004FF400611148FDF778FCB08A48450FD9B9
:1073C000E079401CC0B2E0710A280AD30C48016879
:1073D0000C4A01F4E06111430160BFF34F8FFEE7F7
:1073E000E571BDE8F08700007403002088000020EC
:1073F000280000202004002069020020000C014029
:107400000CED00E00400FA052DE9F84FFF4F0026CF
:107410003546B7F91C30B7F90A20B7F91AC003FB93
:1074200002F1B7F908000CFB02F20CFB001103FBA0
:10743000102041F3CF31F98241F24C4240F3CF307A
:10744000514340F6B8323883424350424318114406
:107450005B10C1F1000134464FEA6102009347D549
:10746000002AB8BF052103DB0028D4BF0421032173
:10747000F9710021E54B797197F807B0B3F90A90DB
:10748000B3F91A10B3F908C0B3F91C8001FB09FA6B
:1074900008FB1CA308FB09F801FB0C8143F3CF3365
:1074A00040F6B83A03FB0AF341F3CF3141F24C4CBA
:1074B00001FB0CF103EB010C5B421944CCF1000C15
:1074C0004910DFF84C934FEA6C0C5B42CCF1000C96
:1074D000C1F1000EA9F1060A40F2EE28BBF1070F38
:1074E00080F0D081DFE80BF0FE0D559EE8FDFC003A
:1074F000002AA8BF0221BBDA0028D4BF062101213F
:10750000B6E7614600F06EFA388DB98D05B20144D8
:10751000B8780EB228B3BAF90000B028A4BF06F1BB
:107520000C0006B20ADA10F1B00FD1BFA6F10C00C0
:1075300040F6B801484306EBE03006B2B9F9000066
:10754000B028A4BF05F10C0005B20ADA10F1B00FA3
:10755000D1BFA5F10C0040F6B801484305EBE0307F
:1075600005B2002EB8BF002603DBB045B8BF40F21D
:10757000EE26002DB8BF002503DBA845B8BF40F2BA
:10758000EE25A9B2B0B200F0DDF90FFA80F800F0F4
:107590007DB91146009800F025FA388DB98D06B2F4
:1075A000084405B2B87828B3BAF90000B028A4BFDF
:1075B00006F10C0006B20ADA10F1B00FD1BFA6F145
:1075C0000C0040F6B801484306EBE03006B2B9F9CA
:1075D0000000B028A4BF05F10C0005B20ADA10F1D2
:1075E000B00FD1BFA5F10C0040F6B801484305EB40
:1075F000E03005B2002EB8BF002603DBB045B8BFAF
:1076000040F2EE26002DB8BF002503DBA845B8BF29
:1076100040F2EE25B1B2A8B200F094F90FFA80F86A
:1076200000F034B90146704600F0DCF9388DB98DB0
:1076300004B20144B8780DB230B3B9F90000B028F3
:10764000A4BF05F10C0005B20ADA10F1B00FD1BFEA
:10765000A5F10C0040F6B801484305EBE03005B257
:107660006C48B0F90000B028A4BF04F10C0004B2CB
:107670000ADA10F1B00FD1BFA4F10C0040F6B80146
:10768000484304EBE03004B2002DB8BF002503DB13
:10769000A845B8BF40F2EE25002CB8BF002403DB9C
:1076A000A045B8BF40F2EE24A1B2A8B200F04AF95A
:1076B0000FFA80F800F0EAB81946104600F092F987
:1076C000388DB98D05B2084404B2B87850B3B9F911
:1076D0000000B028A4BF05F10C0005B20EDA02E0EC
:1076E00080E036E0CEE010F1B00FD1BFA5F10C0084
:1076F00040F6B801484305EBE03005B24548B0F923
:107700000000B028A4BF04F10C0004B20ADA10F1A2
:10771000B00FD1BFA4F10C0040F6B801484304EB10
:10772000E03004B2002DB8BF002503DBA845B8BF88
:1077300040F2EE25002CB8BF002403DBA045B8BF03
:1077400040F2EE24A9B2A0B200F0FCF80FFA80F8E3
:107750009CE07146604600F045F9388DB98D06B25F
:10776000084404B2B87830B3BAF90000B028A4BF16
:1077700006F10C0006B20ADA10F1B00FD1BFA6F183
:107780000C0040F6B801484306EBE03006B2214851
:10779000B0F90000B028A4BF04F10C0004B20ADA6A
:1077A00010F1B00FD1BFA4F10C0040F6B80148436E
:1077B00004EBE03004B2002EB8BF002603DBB04576
:1077C000B8BF40F2EE26002CB8BF002403DBA04572
:1077D000B8BF40F2EE24B1B2A0B200F0B3F80FFA95
:1077E00080F853E01846009900F0FCF8388DB98D08
:1077F00004B20144B8780EB268B3BAF90000B028F8
:10780000A4BF06F10C0006B211DA05E0D00000209A
:107810000A0100201001002010F1B00FD1BFA6F125
:107820000C0040F6B801484306EBE03006B23C4895
:10783000B0F90000B028A4BF04F10C0004B20ADAC9
:1078400010F1B00FD1BFA4F10C0040F6B8014843CD
:1078500004EBE03004B2002EB8BF002603DBB045D5
:10786000B8BF40F2EE26002CB8BF002403DBA045D1
:10787000B8BF40F2EE24A1B2B0B200F063F80FFA44
:1078800080F803E00020F87040F2ED28DFF89490D3
:107890002548DFF898B099F8151069B3DFF890A083
:1078A000F979002301221AF83110FBF7F9FEF87973
:1078B00000230AEBC000012201795846FBF7F0FED5
:1078C00079791C48002901880CBF21F4005141F44A
:1078D00000510180184899F81530011D0A1D002B30
:1078E0000CBF068004800D800CBF148016801348E6
:1078F000A0F80080BDE8F88FDFF844A0F9790023F4
:1079000001221AF83110FBF7CBFEF87900230AEBBD
:10791000C000012201795846FBF7C2FED0E7000003
:1079200010010020500400200024014000280140E4
:1079300050010020202C0140342C0140402C0140FB
:10794000180100202DE9F001DFF894C0012500F1B5
:1079500048039CB240F2EE228CF8035094429EBF42
:1079600040F2ED20BDE8F0017047441AA4B2622C49
:1079700081BF1B3880B2BDE8F00170479FB200F1B3
:107980003D031FFA83F8002440F2DC56A1F11B03EB
:1079900042450ED9F01B80B2904205D98CF80340C5
:1079A000BDE8F00198B270478CF80550BDE8F001D1
:1079B00070479042F2D301F1480087B297423EBF30
:1079C00040F2D320BDE8F001704780B23D3189B26A
:1079D0008A42E3D9301A80B29042E5D9DEE700004E
:1079E000D0000020F0B4274E4FEA21420014C6E92F
:1079F0000A024FF0000144BF02EB6000C6E90A1022
:107A0000F06A002804DAB26A02EB6000C6E90A01F3
:107A1000D6E90A10084440F2EE27B842DCBFF0BCB9
:107A2000704740F2EE2201FB02F3002808BF00215C
:107A300022D000214FF0010C05460A4605E000BFA8
:107A40004000521C4FEA4C0CD2B2984298BF212AF7
:107A5000F6D3420800244FEA5C0C95420CD89342BE
:107A600024BF9B1A61445208601C4FEA5C0CC4B2EC
:107A7000954298BF212CF2D3781AB162F062F0BC23
:107A800070470000D00000202DE9F047524F90B021
:107A90003846FBF783FD514D2846FBF77FFD01215A
:107AA0003846FBF766FD01212846FBF762FD684674
:107AB000FBF776FE4FF4803046114FF4602A4FF00A
:107AC0000109CDE902A600908DF8049000244FF042
:107AD00004088DF805408DF8108069463846FBF79C
:107AE000BBFD6846FBF75CFECDE902A68DF804906D
:107AF0008DF805408DF8108069462846FBF7ACFDEF
:107B00003846FBF748FE2846FBF745FEB94648468F
:107B1000FBF783FD07462846FBF77FFD0742F6D1BA
:107B20000223012200214F464846FBF7E6FD0223CF
:107B30001A4601213846FBF7E0FD02230322082103
:107B40003846FBF7DAFD0223042209213846FBF709
:107B5000D4FD0223012204212846FBF7CEFD022397
:107B60001A4603212846FBF7C8FD022303221946C3
:107B70002846FBF7C2FD0223042210212846FBF70A
:107B8000BCFD01213846FBF72BFD01212846FBF700
:107B900027FD01213846FBF7F6FC01212846FBF7BB
:107BA000F2FC0F4D2846FCF7A9FA0B4806A94C3009
:107BB00005900C4881E811018020CDE90940800042
:107BC000CDE90C640B900E9405A928460F94FCF7A0
:107BD00015FB10B0BDE8F0870024014000280140EB
:107BE000080002406C1100202DE9F04188B007A880
:107BF000FDF753F84FF48050ADF81C0018208DF8B5
:107C00001F00474C03268DF81E6007A92046FCF78D
:107C1000BBFFE114ADF81C1048208DF81F008DF853
:107C20001E6007A92046FCF7AFFFDFF8F88040464A
:107C3000FBF726FF002501248DF816508DF817401C
:107C40008DF818500B208DF819408DF812508DF8D2
:107C500014008DF81A508DF8135002278DF81B5020
:107C60008DF81570ADF8106004A94046FBF792FF3F
:107C70004EF2E046ADF8006041F60C00ADF80200AF
:107C8000701DADF804008DF80A5045F20C008DF817
:107C90000B408DF80C40ADF80600ADF808508DF89B
:107CA0000D406846FBF708FFADF8006042F61C0087
:107CB000ADF802008DF80A40ADF8046042F20C0005
:107CC0008DF80B408DF80C40ADF80600ADF808506B
:107CD0008DF80D406846FBF7EFFE43F20C008DF87F
:107CE0000A70ADF80060ADF804608DF80B408DF8B7
:107CF0000C40ADF80200ADF80600ADF808508DF864
:107D00000D406846FBF7D8FE02214046FBF774FEA3
:107D1000012202214046FBF735FF08B0BDE8F081A3
:107D2000000801400064004010B5002002F0C0F9D6
:107D30000121084602F0C6F9012140F63D6002F03B
:107D4000E5F90121084802F0C9F901210420FCF7F6
:107D500071FF01210548FCF76DFF0121BDE81040CE
:107D6000C803FCF767BF00000700000200023000F4
:107D70002DE9F04D4FF0000846464546FCF72AFD38
:107D8000DFF800B4DFF800A40024ABF80040AAF844
:107D90000040FE48FE4F04803C80204602F0BEFCBE
:107DA0006420FCF749FAFB483C804480F94C0020F1
:107DB0002070FBF7B1FBF84F15E00220FCF70EFA3C
:107DC00028B10220FCF784F92078401C20700221A1
:107DD0003846FBF729FC30B102213846FBF7C6FBD9
:107DE0002078401C207020780228E6D10120FCF782
:107DF00023FAEA49E64B08681F88C0F34A123A445E
:107E00001A8006EB505086B260888988401CC1F306
:107E10004A1180B229448DB260801028C6D318461A
:107E200040F696710088DE4CA0F530502638884226
:107E300003D3E08940F08000E081DA48DB4A4680E5
:107E4000D94805800020014613689B0501D4491CD0
:107E5000C9B2401CC0B2FF28F6D3642901D94FF043
:107E6000010884F80D80E08920F48060E081002022
:107E700002F054FCC7490020CD4F48803888C00725
:107E8000FCD0388820F00100388005E03A88D2071D
:107E900002D0401C4880F4E748880528F6D388467D
:107EA0000A46088945F25001084390805189C04D27
:107EB00041F050010835A8F8061028802E1D3180A9
:107EC000388820F001003880012002F027FC0AE009
:107ED0003888000607D5002002F020FCE08940F435
:107EE0008060E08102E03888C007F1D0002002F015
:107EF00015FC38883B4620F0010038806420FCF7F0
:107F0000A9F91888000603D5E08940F48060E08173
:107F10006420FCF79FF9E08920F40070E0814005BF
:107F20004AD4002002F0FAFB00204146A8F80200E3
:107F30003888C007FCD0388820F00100388005E080
:107F40003A88D20702D0401C4880F4E748880528C8
:107F5000F6D3088944F24002104388804A8942F0EF
:107F60004002A8F8062028803280388820F00100DE
:107F70003880012002F0D2FB0AE03888000607D5DD
:107F8000002002F0CBFBE08940F40070E08102E0C9
:107F90003888C007F1D0002002F0C0FB388820F0FC
:107FA000010038806420FCF755F93888000603D5B5
:107FB000E08940F40070E081002002F0AFFB002077
:107FC0004146A8F802003888C007FCD0388820F065
:107FD0000100388006E03A88D20703D0401CA8F898
:107FE0000200F3E748881428F5D3E08910F4C06F45
:107FF0006FD100224FF490616E48FBF723FB4FF4E2
:10800000E0416C48FBF700FB4FF4E0416248FBF7AE
:10801000FBFA01216748FBF7EDFA01215E48FBF707
:10802000E9FA03216348FBF760FB032301220621E1
:108030006048FBF735FB0323022207215D48FBF76D
:108040002FFB03231A4605215A48FBF729FB3888E2
:1080500020F0010038803888C007FCD0388820F034
:1080600001003880B8F8080044F240010843A8F83D
:108070000400B8F80A1041F04001A8F80610288062
:108080003180388820F001003880012002F046FB62
:108090000AE03888000607D5002002F03FFBE0899F
:1080A00040F40070E08102E03888C007F1D0404819
:1080B000018821F0010101803E4F04213846FBF781
:1080C00055FA01213846FBF75CFB0020A8F80200B6
:1080D0000CE03FE036480088000607D5002002F09B
:1080E0001DFBE08940F40070E08105E00421384682
:1080F000FBF79AFA0028EDD014213846FBF79BFADB
:10810000BBF8002002EB1011ABF800101821384624
:10811000FBF791FABAF8002002EB1011AAF8001050
:108120001C213846FBF787FA01461848028802EB03
:108130001111018004213846FBF718FA0121384655
:10814000FBF71FFBB8F80200401C80B2A8F8020041
:108150001028CBD3002002F0E1FAB8F8080046F26C
:1081600060010843A8F80400B8F80A1047F2600359
:108170001943A8F8061028803180002002F0CEFABA
:108180005D4619E0F2000020F4000020F600002017
:10819000F00000202C000020002801406C1100207D
:1081A00074030020C803002068040020080C01406C
:1081B000102C014000240140BBF80020BAF8001048
:1081C0005746501A00B2002800DA4042464E0FFAD5
:1081D00080FC3088131A1BB2002B00DA5B420FFAC6
:1081E00083F80B1A1BB2002B00DA5B42DFF8FCB0FD
:1081F0001BB245F2757E4FF4804ABCF5A47F15DAB8
:108200004FF4A47CE04511DA63450FDA43F6B86316
:108210009A420BD3994209D3984207D344F24713A9
:108220009A4203D8994201D8984218D9BBF8001055
:10823000714509D12E48008828802E480088388052
:108240002D480088308017E0A5F800A0A7F800A00E
:10825000A6F800A0E08940F08000E0810FE0BBF8C4
:108260000040744508D0224B1A80224A11802249CE
:1082700008802249012008702988514502D32888A6
:10828000C0F50041484661F30F003988514501D3DC
:10829000C1F50041328861F31F40524501D3C2F558
:1082A0000042494662F30F0183B2040C144AA34210
:1082B00000D300141080B2F9003088B2984200DA7E
:1082C0001180B2F900004FF4484148430014108077
:1082D0000C494FF44D425043001408800A4908806D
:1082E000BDE8F04DFCF7BEB9F60000209601002075
:1082F00090010020920100209401002088010020BC
:108300008C0100208A0100208E0100202DE9F84315
:108310006846FCF7C2FCFF20ADF80000DFF84C8196
:1083200000248DF8034069464046FCF72DFC684662
:10833000FCF7B3FC03254E4EADF800508DF803401A
:1083400069463046FCF720FCFF214046FCF76AFCFA
:1083500003213046FCF766FC6846FCF79EFC482784
:108360008DF803704FF4E070ADF8000069463046B8
:10837000FCF70AFC6846FCF790FC4FF4E064ADF8AB
:10838000004018208DF803008DF8025069464046E1
:10839000FCF7FAFB6501ADF8005069463046FCF782
:1083A000F3FB21464046FCF73DFC29463046FCF7EE
:1083B00039FC6846FCF771FCB414ADF800400420A9
:1083C0008DF8030069463046FCF7DEFB2146304657
:1083D000FCF728FC6846FCF760FC4FF40870ADF829
:1083E00000008DF8037069463046FCF7CDFB684607
:1083F000FCF753FC10208DF8030001208DF80200DB
:1084000040F61C40ADF8000069463046FCF7BCFB66
:10841000E400ADF8004069464046FCF7B5FBADF816
:108420000050144D69462846FCF7AEFB002261114E
:108430003046FCF73AFC002204213046FCF735FCBC
:10844000002208213046FCF730FC00221021304683
:10845000FCF72BFC002221462846FCF726FC0122D3
:10846000D1023046FCF721FCBDE8F883000801404A
:10847000000C01400010014038B54FF4A06001F03D
:108480006DFA18208DF8000000248DF801408DF859
:10849000024001258DF80350684601F02DFA19209D
:1084A0008DF800008DF801508DF802408DF80350D2
:1084B000684601F021FA12208DF800008DF8015075
:1084C0008DF802408DF80350684601F015FA1E2021
:1084D0008DF8000002208DF801008DF802408DF823
:1084E0000350684601F008FA14208DF800000320BC
:1084F0008DF801008DF802408DF80350684601F0B8
:10850000FBF9064804800648018821F0010101803A
:10851000018821F08001018038BD00001008004072
:10852000102C0140F0B43D48018801F08F0101801A
:108530004FF4D2710180394A40F2EE212C32118081
:108540000024111F0C80354D012314352B80111D83
:108550000B802E1D46F668013180371D47F66801F5
:108560003980011D4FF47C520A803A1D40F6880C78
:10857000A2F800C0B2F800C04CF4805CA2F800C0C1
:108580000A8822F070020A800A8842F020020A80DB
:108590002A1F118821F080011180DFF880C040F28D
:1085A00077110CF1340CACF800100CF1040CACF8A1
:1085B00000100CF1040CACF800100CF1040C40F2AB
:1085C000ED21ACF80010154945F60C4C4431A1F8EA
:1085D00000C0B1F800C04CF4807CA1F800C0B0F835
:1085E00000C04CF0010CA0F800C0368848F68F702F
:1085F00006400B4806813E8826F0700646810888B2
:1086000040F4004008808120111F08802B801088D2
:108610001480F0BC002002F081B80000002C014062
:108620002C0000203EB54FF6FF70ADF8040045F673
:10863000BF50ADF800004FF40070ADF80600002008
:10864000054CADF802006946204602F015F90121FB
:10865000204602F0EFF83EBD0004004030480169BA
:1086600041F004010161016921F0040101612D4A19
:10867000401510802B494FF6FF702C310880294897
:108680002030018821F001010180264918310B8832
:1086900023F0F3030B800B8843F0F1030B80038876
:1086A00023F00A030380038843F0030303800B884D
:1086B00023F00C030B80038823F0010303800B8855
:1086C00043F003030B80018841F00101018015494B
:1086D00000202831088013490120143108801148F6
:1086E0000830018821F007010180011F0B8843F049
:1086F00080030B80018821F070010180018841F026
:1087000040010180018821F007010180018841F0CA
:1087100004010180108840F00400108070470000C0
:1087200000100240000800404FF0E020016941F0D5
:108730000401016109494FF47A720968B1FBF2F151
:108740004161074AF02182F8141D016941F00101DD
:108750000161016941F002010161704700000020E0
:108760000FE000E070B5234D4FF4906400222146E5
:108770002846FAF767FF00212846FAF73BFF042155
:108780002846FAF7F3FE01212846FAF7AEFF1A4E03
:1087900001213046FAF7A9FFA9142846FAF734FF59
:1087A0000023012206212846FAF77AFF002301223E
:1087B00007213046FAF774FF01212846FAF71AFF1D
:1087C00001213046FAF716FF04212846FAF7CEFEBB
:1087D000012221462846FAF735FF084C01212046A0
:1087E00002F022F82046BDE870400122114602F056
:1087F00039B800000024014000280140002C01404D
:1088000010B5FFF78FFEFFF73FF9FFF727FFFFF7E0
:1088100009FFFFF7ADFAFFF7A5FFFDF7F5FEFFF73C
:108820002BFEFFF7E1F9FFF77FFFFAF775FEBDE8D2
:108830001040FCF755BC0000F0B5334A334BD178FB
:1088400088061AD55889642817D2C90615D4401C41
:1088500080B25881032802D0042805D00DE0D089C9
:1088600040F40060D08108E0FEF736FD2849012081
:10887000C870D07840F01000D070908B0A2802D8D1
:10888000401C908303E02348FF21A0F8C210224D32
:10889000224E234C2F7823480021EFB1D77827F0C0
:1088A0000107D7704170B68A322E02D92678012E80
:1088B00000D0297059788378994208D1217803290A
:1088C00005D09178C07801F00101814203D0D078C1
:1088D00020F00100D070F0BDB58A642D0ED21D7855
:1088E000AD0709D5D57845F00105D5705D7885705F
:1088F000957805F00105C5704170DBE7D17821F06E
:108900000101D170D6E70000740300209404002018
:1089100028000020900200202200002020040020D7
:1089200069020020C80000202DE9F05FDFF800B4E4
:10893000BBF80010BBF80C00814234BF4FF0010AB5
:108940004FF0000ADFF8EC83FB480026A0F11E047C
:10895000B8F80030227820F81230521CD2B22270BF
:10896000042A08BF2670B0F90020B0F902301A447A
:10897000B0F90430B0F90600184410448010A08209
:108980006078EE4FEE4D4FF00309012814D02E739E
:108990006078022818BFA68000F0BE8260780328A5
:1089A0001CBF6078042800F04183E88910F4807FC0
:1089B00000F00B8300F011BBBBF80A00884228BF0F
:1089C000268211D2208A10283CBF401C20820BD363
:1089D00001208BF81E00E88940F02000E88100208B
:1089E00001F09CFE84F80190D6480178012921D03D
:1089F000B8F90220B4F914108A4257DA881A001222
:108A00002E730128B8BF012002DB0428C8BF042050
:108A100082B2B4F904109142D8BFA68007DD081ACB
:108A200000B2A0800028C8BF401E00DDA0802681C3
:108A300000F0FCBA06702E73BAF1000F1CBFB4F937
:108A400004001028C4BF1038A080687B00281CBF19
:108A5000B8F900000B28EADA002001F05FFE607828
:108A6000032818BF6670687B18B1E88940F48070ED
:108A7000E881B548007828B1E88940F00400E88131
:108A800084F801909BF81D0028B1E88940F040006F
:108A9000E88184F801909BF81E000028C7D0E8897F
:108AA00040F02000E88184F80190C0E7E88950B9DF
:108AB000A5480078002801BF9BF81E0000289BF8FD
:108AC0001D00002855D02E73BAF1000F12D0B8F94E
:108AD000001048110428C8BF042002DC002808BF89
:108AE0000120042936DDB4F904108142D2BFA680EA
:108AF000081AA080B8F900000B2802DAB88A962874
:108B000003D9B4F904000A2891DA002001F006FE26
:108B10006078032818BF6670687B18B1E88940F454
:108B20008070E8818848007828B1E88940F0040026
:108B3000E88184F801909BF81D0028B1E88940F095
:108B40004000E88184F801909BF81E0000283FF463
:108B50006EAFA4E7A189491C89B2A1811029CDD3A8
:108B6000B4F904108142C6BF081AA080A680A6816D
:108B7000C4E776480078E0B12E73BAF1000F1CBF4D
:108B8000B4F904000328C4BF401EA080B8F9000057
:108B90001628A4BFB4F904000A28BFF648AF002085
:108BA00001F0BCFDE88940F00800E88184F80190FC
:108BB0003DE7B4F90230B4F90400984203DA0A2B15
:108BC00007DD00F026B90A2BC4BF03F1640181421E
:108BD0007DDCBAF1000F7BD0B98A462979D3B7F989
:108BE00016103A8C914274DB6A7812F0040F1CBFA5
:108BF0002A79002A05D16A7B002A04BFEA7F002A6D
:108C00000BD0534B4FF4007C4FF00102A3F800C08F
:108C10004FF0400CA3F804C012E07B8C4FF0000230
:108C20009942ACBF4FF4807C4FF0800C484BA3F8C6
:108C300000C0ACBF4FF0200C4FF0100CA3F804C0E4
:108C400095F80CC0434BBCF1000F18D14FF00A0C43
:108C5000A4F818C04FEAA11CCCF10009A4F81A909E
:108C6000B3F900C0E14500F3FB81E0824FF0010C55
:108C700085F80CC04FEAC03C3548C0F814C0208BC2
:108C8000002A14BF00EBE10000EB2110C0F100004E
:108C900000B218BF6083B4F91A108142B8BF481CF3
:108CA000C8BF481E00D06083294AB4F91A10B3F92E
:108CB000000000F015FFA080B4F9161040F2DC525D
:108CC0008142C8BF668208DC638A934202E079E091
:108CD0005CE041E09CBF5B1C6382CB1C984202DAE3
:108CE000638A934206D3208B642838BF401C4DD240
:108CF00020834BE0821D8A4206DC218B00291CBFA9
:108D0000491E2183E08241E07A890F2A3ED9E28917
:108D1000521C92B2E281202A38D3E681814235DDAD
:108D2000E082208B002818BF401E2FD0E0E7000013
:108D3000680400208804002086020020200400200F
:108D400074030020D6000020AA010020A801002002
:108D5000E4040020EE0000202E736189491C89B2D2
:108D60006181072912D96681B8F900100B2903DD4A
:108D70000B390911012901DA012102E00429C8BFD8
:108D800004218842A6BF401AA080A680B4F9020040
:108D90000A283FF74CAEB88A462805D9B7F916001D
:108DA000398C88423FF743AEB8F900000B28A4BFC6
:108DB000B4F904000A283FF73AAE002001F0AEFCF7
:108DC000667034E62E736189491C89B261810F296E
:108DD0007FF62DAEBAF1000F18BF98427FF727AE8D
:108DE0006681B8F9001004297FF721AE0B2903DD55
:108DF0000B390911012901DA012102E00429C8BF58
:108E00000421C21A8A42ACBF401AA380FFF60FAEFB
:108E10000CE6DFF854C22E73BCF814C0BCF1780F16
:108E200098BF4FF0080C0FD9DFF83CC2904FBCF848
:108E30000A90DFF838C2B9F10A0F9CF801C017F8A0
:108E40000CC088BF4FEA5C0C6681DFF82892278946
:108E500029F81710791C89B2218161455BD3002163
:108E6000ACF10109B9F1000F16DD834F1CF0010FC1
:108E700008BF37F9021FB7F902B04FF0000A5FEAE6
:108E8000690908D037F904EF5944B7F902B0F24440
:108E9000B9F10109F6D15144BCF1010704D4DFF85E
:108EA000D49139F917703944083191FBFCF1511A0A
:108EB00041F3CF1126810129B8BF012104DB2A89A2
:108EC0008A42B8BFB5F90810674AB2F916C0178BC5
:108ED000BC45A8BF002118DAD28CBA1A624514DA50
:108EE000A7EB0C02521CC2F34F028A42B8BF11B268
:108EF000B8F90020B4F81CC0A2EB0C0C0FFA8CFCE3
:108F0000BCF11E0FC8BF0021A2831A1A9142B4BF40
:108F10000844401CA08089E05848B7F91620006832
:108F2000002AB8BF5242504301F07CFE80B244F6A2
:108F3000E7418842C8BFA18005DCB0F5C87FB8BF53
:108F40004FF4C870A080B5F906000A283BDDE98916
:108F5000C1BBB4F90410884235DB494B01F5FA6016
:108F6000B3F930208242C8BF02461A86454AB2F998
:108F700030308342C8BF108606DC434BB3F9102063
:108F80008242C8BF02461A824048DFF80481466127
:108F90004048C8F814600680FDF758F8F88A0028A1
:108FA00008BFFDF745F8B4F904003B490880C00349
:108FB000C8F8140000F0FEFB01206070A87701F0F3
:108FC000ADFBEBE4FFE76670E8E4617804291FBFBE
:108FD000697B002940F48070E88180B210F0040FB2
:108FE00006D12E49097800291CBF40F00400E88111
:108FF00080B210F0400F06D19BF81D1000291CBF55
:1090000040F04000E88180B210F0200F06D19BF8BC
:109010001E1000291CBF40F02000E8810004000C55
:1090200004D084F80190002001F078FBE88910F466
:10903000885F06D0697B21B930F48850E88108BF89
:109040006670B4F904000028BCBFA680BDE8F09F9C
:1090500044F698118142B8BFA180BDE8F09F00BFDF
:10906000A4F81AC001E600002004002094040020A7
:109070006CCC000858120020561200200802002074
:10908000C803002094030020FA030020FC04002001
:10909000E4040020EA000020EC000020AA010020E7
:1090A0002DE9F0411E4C20781E4B1F4A01280AD0A2
:1090B000D8891E4D10814FF00006E88910F0600F2E
:1090C00003D0D67029E0188AF3E71988B2F808C0EF
:1090D000012761450CD29670D1780F2903D2491C23
:1090E000D170BDE8F0815F7740F04000E881F8E79B
:1090F000D670B3F80AC061450FD99178022902D21F
:10910000491C9170EDE79F7740F02000E881002036
:1091100001F004FB03202070E3E79670E1E7000014
:1091200069020020680400207C00002074030020F5
:1091300010B5FDF72BFAFBF7BDFDFCF703F8FFF7C1
:10914000F3FB00F0FBFFFEF75FF9FCF72FF9BDE83A
:109150001040FBF70DBEFCF763BA000006498968B2
:10916000C90941430A20B1FBF0F004490988B0FB6A
:10917000F1F080B27047000050040020200400206D
:109180002DE9F041294C208B1E2801D800200CE04D
:10919000322801D8052008E0642801D80A2004E01C
:1091A000962801D80F2000E01420E0840A20FFF761
:1091B000D5FFE0831E48408EFFF7D0FFA084E08BF0
:1091C0004FF6FF71C0EBC000208401EA40006084CC
:1091D00018483C211A4F007DB1FBF0F0A0851648DD
:1091E00016490278C87862F3C300C870A48AB4B183
:1091F000B868401CB860012811D002F063FC054635
:109200000E46F86802F05EFC0E4A0F4B02F06EFC50
:109210002A46334602F08AFA02F010FCF882388BB4
:10922000A04200D23C83BDE8F08100002004002071
:10923000900200205004002022000020740300202F
:10924000A0040020CDCCCCCCCCCC0C402DE9F047F8
:109250003D4F64213888484302F034FC3B4A3C4B84
:1092600002F064FA02F0EAFB3A4C86B2BE80B4F92E
:1092700000000025DFF8E080DFF8E090002816DD30
:1092800000EB8000400002F01DFC354A354B02F037
:109290004DFA02F0D3FB80B26081282808D998F8F3
:1092A000000005281AD2401C88F8000002E0658101
:1092B00088F8005060892C4D46434FF47A7096FB35
:1092C000F0F0F8802878294C80064FF4806108D5AA
:1092D00001222046FBF7E9FC012207E089F81F5034
:1092E000E8E700222046FBF7E0FC002208212046A8
:1092F000FBF7DBFC99F80D00B8B11C4D0835286868
:10930000400701D5002200E0012204212046FBF79E
:10931000CCFC2868C00601D5002200E001222046CE
:10932000BDE8F0471021FBF7C0BC2878800605D5C2
:10933000012204212046FBF7B8FCEFE700220421BC
:109340002046FBF7B2FCE7E76804002027A74D841E
:109350003CE07E4088040020C80000207403002008
:10936000888E55636DE35D4094040020000C01403D
:109370002DE9F84FFB48FC4A0A210688B0F802A004
:10938000108EFB4BB0FBF1F0F8494883202183F8A5
:1093900023108946F749C0B22D2881F8220003D94D
:1093A000F4482D2180F82210EF48F34CB0F8B200B9
:1093B00048B9ED48B0F8B61029B190F8B10010B135
:1093C00020720F2801D90F202072EC480078642504
:1093D00020B96E2E02D8EA48007820B1207A00EB3E
:1093E00080008000F3E0E748C078C0076FD1E6480E
:1093F0004778781E09286AD2DD48DFF874B3C0794F
:109400000BF1240BE8B3DA4A44F69813114601280D
:1094100091F82D1001FB03F85AD0022874D0207A5D
:109420006421484302F04EFBD84AD94B02F05EFB60
:109430000022D84B02F07AF902F000FBCC49888177
:10944000B8FBF5F0A1F80890C885DFF828834146FD
:1094500001F1190098F8002023310091002A75D0FD
:10946000434603F10F0193F82C3044F6981C03FB9C
:109470000CFB012A70D0022A67D0207A642148436D
:1094800000E01CE002F01EFBC04AC14B02F02EFBC4
:109490000022C04B02F04AF902F0D0FAA8F8060008
:1094A00098F82200A8F80200BBFBF5F0A8F82E00FF
:1094B000B448007900287CD0B8F8060094E0AC48A5
:1094C000DFF8AC821A30395CA8F8081020E07AE0A6
:1094D000A749A2F808901031207A795C9346484356
:1094E00002F0F0FAA94AAA4B02F000FB0022A94BB5
:1094F00002F01CF902F0A2FAABF80C00B8FBF5F090
:10950000ABF82E00A1E7FFE7DFF86482A8F8089027
:10951000207A6421484302F0D5FA9C4A9C4B02F021
:10952000E5FA00229B4B02F001F902F087FAA8F855
:109530000C0017F80B0044F698114843B0FBF5F007
:10954000A8F82E0081E701E006E01BE0395CA8F8EE
:109550000210207A64211AE098F82220A8F802204C
:10956000207A795C484302F0ADFA884A884B02F0D1
:10957000BDFA0022874B02F0D9F802F05FFAA8F892
:10958000060091E73A5CA8F80220207A795C48430B
:1095900002F098FA7D4A7E4B02F0A8FA00227D4B39
:1095A00002F0C4F802F04AFAA8F806000098385C05
:1095B00000E005E044F698114843B0FBF5F075E78C
:1095C0006B48808910E0207A00EB8000400002F0B8
:1095D00079FA6E4A6E4B02F089FA00226D4B02F066
:1095E000A5F802F02BFA80B261490A89202A01D934
:1095F000A1F808905F494A8891F822108A4201D95F
:109600005C4A518064490978644FDFF894C10129AC
:10961000BA8808D1BCF80A1029B18A4206D21E299C
:1096200004D91E3911E0ACF80A2010E08A4203D2B6
:109630000A2901D90A3908E08A4203D2052901D949
:10964000491F02E08A4202D2491EACF80A1046497C
:10965000B1F8C21064290ED80A2920D2022912D3E7
:10966000A0F1EF02891E5143CA1701EB5271EF229C
:1096700002EBE10111E0BB8ABCF80A2093420ED94B
:10968000F98A914201D9EF210AE05B1A511AA0F13F
:10969000EF02514391FBF3F1EF3109B200E001B267
:1096A000304B64271A88A2F15F0808FB07F95F882E
:1096B00064226E3F07FB02FB6E2E02D8BAF1820FC6
:1096C00001D9EF2017E05F2E02D8BAF16E0F11D941
:1096D0000FFA88F23BB29A4203DB0F2399FBF3F2B5
:1096E00002E014239BFBF3F2A0F1EF035A43B2FB19
:1096F000F5F2801A00B2814200DC0846A080207A90
:1097000002F0E0F9274A284B02F0F0F90022274B3B
:1097100002F0ECF94FF0FF3202F0B1FD02F05EF919
:1097200000B26E2E02D8BAF1820F01D9002011E0EA
:109730005F2E02D8BAF16E0F0CD9B84503DB0F22A9
:1097400099FBF2F102E014229BFBF2F14143B1FBE1
:10975000F5F1401AE08007481549C08DC881BDE881
:10976000F88F00001A000020900200202004002042
:10977000C80300209403002088040020A9010020D1
:10978000A80100207403002094040020888E5563F3
:109790006DE35D400000594069020020680400202C
:1097A00094000020581678658157564000001C40F0
:1097B000FA0300202DE9F041404E414C414DF08D1F
:1097C0002080E87B08B106202881B6F8B2003E4F21
:1097D0004FF6FF7210B9B6F8B60090B128896FF055
:1097E000040100EB800001EB400080B2FFF7B6FC03
:1097F0006881788800EB800002EA4000FFF7AEFC49
:1098000014E096F8BB0000EB4001C1EBC01002EA87
:10981000C00000F065F8688196F8BB0000EB4001DD
:10982000C1EBC01002EAC00000F05AF8B880274827
:10983000274A0188208B1268504301F0F3F9622116
:1098400048436421B0FBF1F044F69811884203D8F4
:109850004FF44871884200D208461E4A50811E4883
:1098600000781E4B4FF47A7101280CD0D8780F285D
:1098700004D8401CC0B2D8700F2806D3A08B8842F1
:1098800015D2401D12E00020D870D078C00701D05A
:10989000708E0BE0107920B1788800EB80004000DA
:1098A00004E0288900EB80004000401FA0830004F2
:1098B000000C00D1A183BDE8F081000090020020DF
:1098C00020040020C8030020940300206804002026
:1098D0000802002074030020690200209400002088
:1098E0000349C96841433C20B1FBF0F080B27047A6
:1098F00050040020FEE7704730B50F23C27801788E
:109900000125F2B1144A126801F1E02102F4E0628B
:10991000C2F5E062120AC2F10404D3404278A240C8
:1099200084781C401443220181F80024007800F060
:109930001F018D404009800000F1E020C0F8005177
:1099400030BD01F01F0085404809800000F1E02093
:10995000C0F8805130BD00000CED00E00249084322
:1099600002490860704700000000FA050CED00E0B5
:10997000024A1140014302480160704780FFFF1F07
:1099800008ED00E070B5144A09200021108013484A
:109990000469436823441D0C558093800368234465
:1099A0001C0CD480138183681C0C54819381008B20
:1099B000D081002032F81030401C194480B289B2A6
:1099C0001328F7D3D18414220349054800F066FC1C
:1099D00004490020887070BD1C100020A0040020E5
:1099E00000E800082800002070B53648364C818A0F
:1099F000207B232901D9012802D840F2262114E036
:109A00003C2901D9022802D84FF4E1710DE05A290E
:109A100001D9032802D84FF4AF7106E0782901D9A3
:109A2000042801D8FA2100E0C821284A1268284DEC
:109A300002F020024FF6FF762A80AB88B34201D2B3
:109A40005B1CAB8000235AB96E884EB1AE8866812C
:109A5000AB80FF2804D2401CC0B22073012812D072
:109A60006689A888864200D860816A806089012260
:109A7000884203D21749B1F8501031B123812373C2
:109A800084F8322070BD5020EEE7022801D212483F
:109A900002E01249B1FBF0F06421B0FBF1F00004E8
:109AA000000C208100D12281207B617B401C8842F8
:109AB00001D384F832302089C828E3D9C820208116
:109AC00070BD00002004002094030020080C014019
:109AD000660000209002002090D0030020A1070023
:109AE00030B4081AB2F90010136901FB00FCB2F996
:109AF000041048435169C417081844EBE1714FEA58
:109B0000E3741D1A8C4106DBD368DC17C51AA1412A
:109B1000A8BF506101DA184653616044B2F90A10D7
:109B2000C0138142AABFB2F9081008468142C8BFDB
:109B3000B2F9080000B230BC70470000164900209E
:109B4000C989CA0701D18A0701D5032021E04A0744
:109B500001D504201DE0CA0601D5432019E08A067C
:109B600001D5D02015E00A0603D48A0501D44A05A0
:109B700001D541200DE0090501D5802009E0074904
:109B80000A886E2A01D3A12003E04988822900D3E4
:109B9000A620034908727047740300201A000020B1
:109BA000940400202DE9F04F4A4A4FF0030B4A4835
:109BB00082F801B0494A00F80DBF0F24484B1472D7
:109BC00002229A70474B4FF00109FA22A3F8129033
:109BD0009A824FF0C80AA3F816A04FF4C8721A83ED
:109BE0004FF496725A8340F28A229A834FF4C872D5
:109BF000DA8352001A844FF4FA725A84394A40F2D6
:109C0000B633142593840A238370C5701E22027113
:109C100028224271322282713C26C6714627077281
:109C20004FF0500880F809804FF05A0C80F80AC0B5
:109C30006422C2728375C6754126067647764B2626
:109C4000867680F81B805526067780F81DC05F2633
:109C50008677C2770C220273002142730D22827331
:109C6000C473112202741222427485741622C274C3
:109C70001722027519221C4D42750324AC701B4C2F
:109C800000F80D9D1A4D628342186C18D67B26741D
:109C900092F8236084F82460491C527EC9B2A276EF
:109CA0000A29F1D3134885F807B00621A0F812A0BD
:109CB0000175437040F2DC5101824FF42071C18084
:109CC0000D49002008800D4908808870C870BDE8E3
:109CD000F08F00007403002094030020880400200B
:109CE00068040020FA0300209404002020040020CF
:109CF000C80300205004002014000020160000209B
:109D000070B54E4D4E490024A8784870A8880F2899
:109D100002D900204B4901E001F0D4FE01F08EFE93
:109D2000494908724949A8798870494805EB4401B6
:109D300000EB4402641CB1F86410E4B251820A2CB6
:109D4000F4D3444A002005EB40011318401C91F85D
:109D5000C810C0B2D9730A28F5D3002005EB400122
:109D60001318401C91F8DC10C0B259760A28F5D3BC
:109D7000002005EB4001B1F8F010642900D96421FE
:109D80001318401CC0B283F823100A28F1D33249BB
:109D900095F80401887095F80601507395F808014C
:109DA00010702E4A002005EB40011318401C91F85A
:109DB0002C11C0B219740A28F5D3002005EB40011C
:109DC0001318401C91F84011C0B299760A28F5D3B7
:109DD000002005EB4001B1F85411642900D9642139
:109DE0001318401CC0B283F824100A28F1D395F848
:109DF00068011B49D071B5F86A0148831948B5F864
:109E00009011418295F89211017595F89411417065
:109E1000B5F896110182B5F89811C1801249B5F8CC
:109E20009A0108801148B5F89C11018095F89E119F
:109E3000817095F8A011C17070BD0000DC09002090
:109E40007403002000002E408804002068040020D5
:109E5000FA0300209403002094040020C80300208B
:109E600020040020500400201400002016000020D0
:109E700070B5534A00210C2010805248544B407852
:109E800050805148007A908050488078D0800846B1
:109E900003EB400402EB4005401C648A80B2A5F845
:109EA00064400A28F4D34B4B00201C1802EB4005F9
:109EB000401CE47B80B2A5F8C8400A28F5D30020F6
:109EC0001C1802EB4005401C647E80B2A5F8DC4003
:109ED0000A28F5D300201C1802EB4005401C94F81A
:109EE000234080B2A5F8F0400A28F4D33A4880789D
:109EF000A2F80401587BA2F806011878A2F808011C
:109F0000364B00201C1802EB4005401C247C80B21C
:109F1000A5F82C410A28F5D300201C1802EB4005B7
:109F2000401CA47E80B2A5F840410A28F5D3002049
:109F30001C1802EB4005401C94F8244080B2A5F8A0
:109F400054410A28F4D3D879A2F868012448408BF8
:109F5000A2F86A012348438AA2F89031037DA2F84F
:109F600092314378A2F89431038AA2F89631C088DE
:109F7000A2F898011C480088A2F89A011B4803889F
:109F8000A2F89C318378A2F89E31C078A2F8A00193
:109F900000204FF4C77332F81040401C214480B2B7
:109FA00089B29842F7D9A2F81E134FF4C872044937
:109FB0000F4800F073F90F490020087070BD0000D1
:109FC000DC090020740300208804002068040020BD
:109FD000FA0300209403002094040020C80300200A
:109FE000200400205004002014000020160000204F
:109FF00000E0000828000020254810B5B0F8C44053
:10A000002448254A0023B0F90000B2F9301054B9B1
:10A01000148944B1947B34B192F832401CB91F4C7E
:10A02000E478E4060AD5814200DD1086B2F93000FA
:10A03000802801DD803828E0138610BD184C81424D
:10A04000237000DA108617498B8A502B02D9B0F59D
:10A05000FA6F04DA144880788000001D07E0488910
:10A06000202801D9202002E0082800D20820B2F9D7
:10A0700030304FF4C8718B4200DA1186B2F93010DB
:10A080000844D18D884200DB88B2108610BD0000E4
:10A09000900200206C020020940300207403002032
:10A0A00022000020200400209404002070470000BB
:10A0B000034A516821F44041014351607047000058
:10A0C00000100240044A0029516901D0014300E018
:10A0D000814351617047000000100240044A00298A
:10A0E000D16901D0014300E08143D1617047000094
:10A0F00000100240044A0029116901D0014300E028
:10A10000814311617047000000100240044A002999
:10A11000916901D0014300E08143916170470000E3
:10A1200000100240044A0029D16801D0014300E038
:10A130008143D160704700000010024070B5FBF70A
:10A14000BFF9494A49484FF0010CB2F91A10B0F969
:10A15000000001FB01F4002812DD884226DD4043A7
:10A16000031B002010214D1E0CFA05F10E18B1B290
:10A170004943994298BFB0B215F0FF01F3D115E001
:10A1800018BF884212DA4043031B00211020401EF2
:10A190000CFA00F50D44AEB276439E4298BFA9B2C8
:10A1A00010F0FF00F3D14842908300E090833048E4
:10A1B000304B4FF00005C07810F0010F2BD1B2F9F1
:10A1C0001C0000FB00411C78012C24D1182922DD41
:10A1D000B1F1805F1FD228490978E1B92749098880
:10A1E0000C2903D8264909880C2914D99178A1B1E2
:10A1F000B0F5804FC8BF40F2651006DC40F2651133
:10A20000484380131128B8BF1120B2F91E108142B3
:10A2100019DA1079B8B1957015E0B0F5804FC8BF64
:10A2200040F27D3006DC40F27D31484380132C281B
:10A23000B8BF2C20B2F91E10814204DD107900282D
:10A2400018BF82F802C01878042828BF70BDDFE864
:10A2500000F002090202002000F060FABDE8704040
:10A26000FBF74AB970BD0000D00000206C0200204E
:10A2700074030020690200209D010020BE0100201F
:10A28000C001002010B5002305E030F8024B21F892
:10A2900013405B1C9BB29342F7D310BD2DE9F05FD6
:10A2A000A0F10064154688468246B4F5803F50D23E
:10A2B000FAF72EFBA70AC4F34806C6F50074A542B8
:10A2C00000D82C46DFF890B04FF0006000EB8720FC
:10A2D00081464FF400722049FFF7D4FF00204FF66B
:10A2E000FF7206E033183BF81310914203D1401C73
:10A2F00080B2A042F6D3A04223D24846FAF7ACFA85
:10A3000000205A4606E038F810108319401C22F845
:10A31000131080B2A042F6D348464FF400720E49A3
:10A3200000F01CF8A54210D0281B08EB4408A244FA
:10A33000002685B24FF400747F1CA542C4D82C4679
:10A34000C2E7224641465046EAE7BDE8F05FFAF729
:10A35000B9BABDE8F09F0000DC0500202DE9F0410E
:10A3600016460F460546FAF7D3FA2846FAF774FA66
:10A3700004280BD1002407E037F814102846FAF718
:10A38000A9FA641CA4B2AD1CB442F5D3BDE8F041F7
:10A39000FAF798BA704700001D48016841F480310F
:10A3A000016001688903FCD51A490A6842F010026D
:10A3B0000A600A6822F003020A600A6842F0030297
:10A3C0000A6041684160416841F440514160416820
:10A3D00041F4C0614160416821F47C1141604168F1
:10A3E00041F424114160016841F08071016001680D
:10A3F0008901FCD5416821F003014160416841F0C9
:10A40000020141604168C1F381010229FAD170471C
:10A4100000100240002002402DE9F0413D4E3E4F29
:10A42000F08A10B142F2107004E0387D01281DD08E
:10A430004FF47A7039493A4DDFF8E880CA88E988E4
:10A4400000244FF6FF73B2F5E16F1DD2AA88824255
:10A4500001D2521CAA8092B2012A0AD0824203D3AE
:10A46000EC602C617380F3802C811DE040F6B830E5
:10A47000E0E7814202D20120287003E0002140463B
:10A4800000F0F8F9EC80EFE72A890A2A02D2521C80
:10A490002A8100E0AC80814202D2491CE98003E0BD
:10A4A000EC602C617380F3802878002830D0B08A6B
:10A4B0003228404608D800F0CCF9C5E90304397DBC
:10A4C000414371806C7013E000F0C3F92969401AB0
:10A4D000E860084428616878401CC0B26870397D23
:10A4E000884209D36C7040462C6100F0B2F970804C
:10A4F0000021404600F0BEF9387DA9894843F0802C
:10A50000387820B1B878052801D2401CB8702C707A
:10A51000BDE8F08120040020500400201A00002033
:10A5200094000020000400402DE9F007DFF850916E
:10A53000544DB9F90020B5F906709742B8BF3A46B4
:10A540004EDB514B00EB900C8C45B3F9003011D829
:10A550009A427DDC0A2838BF802004D3081A80B2D2
:10A56000042888BF04208242CCBF101A00226DDD6F
:10A5700002B26BE000EB400C444C0CEB001CA4FB63
:10A580000C4C4FEA1C14DFF808C1424E4FF0000893
:10A59000BCF900C0A14213D29A4268DBB5F90A00A7
:10A5A0009042C8BF024651DC308800F5807000B28E
:10A5B00030808445DCBFA6F80080501C46DCD7E71D
:10A5C00081420ED29A4254DB7088403000B27080D3
:10A5D000604503DB501CA6F8028002B2A6F8048096
:10A5E00034E033D92C4C4FF47A7CE48B00EBC40A72
:10A5F0008A4538BF4FF0010C12D300EB840A8A451C
:10A6000038BF4FF00A0C0BD300EB440A8A4538BF21
:10A610004FF0320C04D32044884238BF4FF0640C12
:10A62000E87F002818BF4FF0140C9A4223DCB08852
:10A63000401C00B2B080844506DCA6F80480002AE5
:10A64000C6BF501E02B20022A6F80280974200E068
:10A650000BE012DB44F698108242C8BF44F6981211
:10A66000A9F80020BDE8F00770471A4672E71A46BD
:10A6700094E71A46A8E71A46D9E73A46EAE70000FF
:10A680006A020020740300206C020020CDCCCCCCE8
:10A69000EE0000205000002020040020014901208D
:10A6A00008707047620300200C48016841F0010106
:10A6B000016041680A4A114041600168094A11403D
:10A6C0000160016821F480210160416821F4FE01EC
:10A6D00041604FF41F018160FFF75EBE0010024031
:10A6E0000000FFF8FFFFF6FE10B58021084800F0DB
:10A6F0009EF8002000F012F8FAF7FEFE0548C18926
:10A7000041F01001C18104490320087010BD000010
:10A71000002C01407403002069020020054A1188C2
:10A720004FF6AA23194010B140F255500143118051
:10A7300070470000202C014010B501210D4800F0A9
:10A7400073F8FEF7F5FC0220F9F748FD00280FD05A
:10A7500002210948F8F768FF002809D002210748BC
:10A76000F8F762FF002803D0BDE81040F8F7D4BE28
:10A7700010BD0000002C01400024014000280140D1
:10A7800010B510218C06204600F065F898B1102114
:10A79000204600F04CF8204600F058F8094A51884D
:10A7A000884201D9411A03E04FF6FF73591A014458
:10A7B0001180508010BD2046BDE81040012100F0FE
:10A7C00033B800006C00002070B5144D01212846FC
:10A7D00000F041F860B10121284600F025F810484A
:10A7E000818C2D2928BF70BD818C491C818470BD4E
:10A7F0000221284600F018F80A4C208820F00200B8
:10A800002080FBF72BFC208840F0020020802846A7
:10A81000BDE87040022100F007B8000000080040C9
:10A82000980100200C080040C94301827047C943C9
:10A83000018270470029018802D041F0010101E046
:10A8400021F0010101807047808E7047B0F8400010
:10A850007047808C704702460020128A0A4200D05E
:10A8600001207047002A828901D00A4300E08A4310
:10A87000828170478184704730B502881B4C1C4D23
:10A88000A0420DD0A8420BD0B0F1804F08D0194B98
:10A89000984205D0184B984202D0184B984203D1E9
:10A8A00022F070034A881A43154B984206D0154B84
:10A8B000984203D022F44073CA881A4302808A88DF
:10A8C00082850A880285A0420AD0A84208D00E4A92
:10A8D000904205D00D4A904202D00D4A904201D1DB
:10A8E000097A01860121818230BD0000002C0140DF
:10A8F000003401400004004000080040000C00400B
:10A90000001000400014004000400140004401409D
:10A910000048014070B5414D2878002876D00024C9
:10A920002C70E878401CC0B2E870012812D1EC709D
:10A93000FCF74AFCFFF758F8FFF76EFDF9F730FA1D
:10A94000FAF7C4FAFBF7A0FA00F0EAFCF9F78EFC7C
:10A9500000F042FA6879401CC0B26871052806D13F
:10A960006C7100F099F8F9F761FA00F0C5FDA8796B
:10A97000401CC0B2A8710A2800D1AC71E879401C13
:10A98000C0B2E871322806D1EC71FCF74DFCFEF73D
:10A9900087FBFFF7D3F8287A401CC0B228726428DE
:10A9A00006D12C72FAF7B0FBF9F76CFAFCF7A8FCA9
:10A9B0006889401C80B26881B0F5967F0AD16C81AD
:10A9C000FEF744FCFEF7D4FCFEF7F4FEFAF77EFC3B
:10A9D000FAF796F8A889401C80B2A881B0F5FA7FF2
:10A9E00006D1AC81FDF728FFFAF7A2FDF8F7E2FEE9
:10A9F000E889401C80B2E881B0F57A7F06D1EC810D
:10AA000000F00EF8FEF7BCFBF9F71EFBFBF7DCFFCE
:10AA1000FCF7DAFABDE87040FAF7D2BA6203002018
:10AA200070B51A4C0021A08800F05CFA21888142A0
:10AA300001D2491C03E019B1814201D9491E21808C
:10AA4000E088134DB0F5E16F03D9012100F04AFA17
:10AA5000E8806088E988884201D2401C03E018B190
:10AA6000884201D9401E608020880A4A00EB80009D
:10AA70004FF6FF7101EA400022F84C0F608800EBAE
:10AA8000800001EA4000508070BD00001A000020E4
:10AA9000C8000020900200202DE9F0412A484078AB
:10AAA00040074FD529482B4D294C028928882A4B2D
:10AAB00042B12178012905D19988C831884201D94C
:10AAC000998000E098809E88B6F5596F00D20026E4
:10AAD000217821480129C06809D142B140F63541A9
:10AAE00071431E4CB0EB411F01D302D808B94FF09F
:10AAF0000504A0FB04011A4F98463A464FF00003A4
:10AB0000F8F782FB391B714341181648B1FBF0F08E
:10AB100080B26880B0F52F7F01D800200FE0B0F53B
:10AB2000616F02D341F2883009E041F28832A0F52A
:10AB30002F70504340F6543290FBF2F080B2E88020
:10AB4000C8F80C10BDE8F0817403002094030020C5
:10AB500069020020FA0300206C000020AC84010090
:10AB6000A0860100EB9207007047000010B5064C6C
:10AB700040F22551204600F009F82046BDE810407B
:10AB800040F2277100F002B80044004070B501F0B7
:10AB90001F0501260024C1F3421306FA05F2012B1A
:10ABA0000FD0022B0FD0838A4FEA11210088134265
:10ABB00006FA01F600EA060001D000B101242046A1
:10ABC00070BD8389F0E7038AEEE7000010B5114AF3
:10ABD00000211148F9F752F80E48017A042914D1DE
:10ABE0000C4C40681E3C010A60702170C0F30D409F
:10ABF000608004F1290000F0CFF8207800210528BA
:10AC000004D0032801D10548418110BD0448818347
:10AC100010BD00008805002000640040940400205E
:10AC200074030020002904BF0020704730B40023C3
:10AC30004FF0010C0D461A4605E000BF4900521CBA
:10AC40004FEA4C0CD2B2814298BF212AF6D34A086F
:10AC500000244FEA5C0C95420CD8904224BF801A25
:10AC600063445208611C4FEA5C0CCCB2954298BF19
:10AC7000212CF2D330BC18467047FEE7F0B51F48D0
:10AC800000211F4A41704FF6FF70908050801D4890
:10AC90001F4A5F2341751C48214C81731B48E60302
:10ACA00081721C48917303806E23438042F20F70BF
:10ACB000508119484FF48072202301741748028094
:10ACC000012242808380C28004819503458153071D
:10ACD000C660C0E90431134897020780428080278C
:10ACE0008780C28004814581C660C0E904310E4876
:10ACF000FF2120F8AC2FC182F0BD00009404002099
:10AD00002004002050040020C8030020FA03002083
:10AD1000940300201A00002074030020E4040020A3
:10AD200000C0FFFFFC04002090020020154810B571
:10AD3000002200F8022F0123427083700421C170A9
:10AD400003210171427182710FA1C2710C6804620A
:10AD50004C684462098901850E494FF6FF74498B9E
:10AD600001EB810104EA4101C185022180F8A310B1
:10AD7000A0F8B0304FF42F71A0F8BC10A0F8C2209A
:10AD800010BD0000900200205A4552585F43414ECA
:10AD90005F310000200400201CB501788C0901F00F
:10ADA0003F018DF800408DF804104278837802EB63
:10ADB0000322084B92B21B7806D0012C07D0022C3C
:10ADC00001D100F07DF91CBD00F020FA1CBD00F09F
:10ADD000E1F91CBD6A050020F8B51E4EF07A002886
:10ADE00020D0B1883289881A83B2304600240068A6
:10ADF0001AB1072B17D9072516E0164A0529C9B23B
:10AE0000D2884FF00003009203D8002200F008FC23
:10AE10001DE0012200F004FCB088052800D90520BF
:10AE20003081B472F8BDDDB210440094B37A0222CE
:10AE3000294600F0F5FB3089284480B23081B17A90
:10AE4000491C01F00F01B172B1888842EAD3F47253
:10AE5000F8BD000014050020094A002101EB410360
:10AE600032F81330834204D101EB410002EB400081
:10AE70007047491C89B22C29F0D30020704700008C
:10AE80000AC3000814488078C2071448C1880CD04F
:10AE900040F2DC52808A914217D9104A40F6AC53F6
:10AEA0009942928C07D310460FE00D4A527800EB7E
:10AEB0004200408A09E0121AA1F2DC535A434FF4CF
:10AEC000FA6392FBF3F2104480B241434FF47A707C
:10AED00091FBF0F000B2704774030020FA030020E9
:10AEE00094040020002247F6F813984284BF002003
:10AEF000704730B401230E4C04F5217500290CBFB6
:10AF000054F822C055F822C0844504D3521C5B1C5F
:10AF100092B2A22BF2DD00291EBF104630BC704752
:10AF2000282A86BFA2F1280080B2002030BC7047DA
:10AF300064C700082DE9F04F574B0027574DB3F871
:10AF400008C04FF4FA61BCF1000F1DD06F81B5F954
:10AF50000600DFF84CA1C0EB8012544CBAF9000097
:10AF6000DFF84091104480112881B5F80A808B46A3
:10AF70004D4EB4F91010A289B9F81400D8450BD27F
:10AF8000BCF1000F06D008E068898842DFD2401C7F
:10AF90006881DCE73C2800D382B194F80AC0BCF198
:10AFA000000F0BD093F8323003B13AB1404AD27857
:10AFB000D20603D43F4AB2F8C42072B1B6F90000F9
:10AFC000814200DD2082B4F91000B0F5807F02DDFF
:10AFD000A0F5807055E0278254E04FF4C87291428A
:10AFE00000DA2282FFF74EFF334980B220810F70D2
:10AFF000B5F90810884225DDA0EB0100B9F80A2058
:10B000002E49C0F38F000A2A02D94978183103E08B
:10B010004A78082101EB5201814200D20846B4F976
:10B020001020B6F900108A4200DA2182B4F910101B
:10B03000594503DA4FF6FF7202EA800000B9012099
:10B04000084415E017DA081AC0F38F00082801D960
:10B05000082001E000B90120B4F91020B6F9001071
:10B060008A4200DD2182B4F91010814202DD081A03
:10B07000208200E02782B4F91000E189884201DDD6
:10B0800088B22082A08908B1401EA081BAF80000D1
:10B09000E880BDE8F08F0000940300206C000020E1
:10B0A000EE000020200400206C020020FA030020A3
:10B0B000740300209002002022000020940400204D
:10B0C00070B5314D95F84720002A5BD095F84620A1
:10B0D0008A4251D1B5F84010B5F84230C91A8AB247
:10B0E000072A01D9072400E0D4B22B44411C224690
:10B0F0001846F8F700F9B5F84200204480B2A5F8E8
:10B10000420095F84610491C01F00F0185F84610E1
:10B11000B5F84010884235D3B5F84400FFF79CFEDF
:10B12000040029D0E07838BBA0881849B5F8402041
:10B13000461815493046F8F7DEF8B5F84000A17812
:10B14000884204D2091A30442022F8F719F9B5F8D8
:10B150004400042806D0A0F58071573902D0B0F51C
:10B16000AC7F02D10A4A0121D17095F8483095F898
:10B170004020054900F0B4FABDE870404A21024879
:10B18000F8F706B970BD00002005002090020020ED
:10B19000280000202DE9F047814698460F461646C4
:10B1A0001046FFF759FE05002CD0174C94F84700C5
:10B1B00018B14A212046F8F7EBF8A978B81E891C87
:10B1C0003E281FD28F421DD880B2A4F84000052827
:10B1D00001D9052100E0014624F8421F00216680C4
:10B1E00021710121617184F8068000280AD00528A8
:10B1F00000D9052009F10301BDE8F047C2B20248B9
:10B20000F8F779B8BDE8F087200500202DE9F05F58
:10B2100007469B460D4616461046FFF71DFE0400E6
:10B220003DD02C4890F8470018B14A212948F8F73A
:10B23000AFF829494FF000094FF0010A022D1CD048
:10B24000E07800282BD1AD1EA078EDB2A84200D244
:10B250000546A0882A4608448046F91CF8F74BF8B2
:10B26000A078A84205D9411B08EB05002022F8F779
:10B2700087F8B6F5887F14D024E0A08801441548EB
:10B280000C380160A1788180C680A0F8089013492D
:10B2900080F80A9080F80BA081F801B08E80BDE89C
:10B2A000F09F0F4A907868B90E48A0F81890C0F83F
:10B2B0000890046943682344C0E90093C0F81090E3
:10B2C00082F802A05B462A46F91C3046BDE8F05FD2
:10B2D00000F006BA20050020900200204000002067
:10B2E00028000020A004002072B64FF440514FF017
:10B2F0000060FEF73DFBFBF7FBFFFFF7BFFCFFF72E
:10B3000015FDF9F723FBF8F7B5FAFDF779FAF9F728
:10B3100042FE62B6F9F74CFEFFF7FCFAFCE70000CC
:10B320002DE9F04F6A4F0122B7F802A0BAF5BA5FD3
:10B3300038BFBA73674801896748B0F8068031B9E9
:10B340006448B8F1640F8273634838BF82724FF06B
:10B35000000C6249624D81F800C081F801C081F89B
:10B3600002C028785F4B604C0128B3F916B09E8A62
:10B3700007D00A2E05D8BBF10A0FDCBFE27784F8AC
:10B380001EC05A4890F8009049F0400980F800909B
:10B3900095F800E05648BEF1000F04BFB4F80EE087
:10B3A000BEF1000F7ED1B4F906E0BEF10A0FA4BFD2
:10B3B00094F80DE0BEF1000F7CD1B3F818E0AEF1C7
:10B3C000050EF34576DA94F803B01BF0100F71D137
:10B3D000DFF820E1BEF8C4E0BEF1000F6AD19B8B1C
:10B3E00006F11E0E9E4565D21BF0010F4FF0020BB9
:10B3F00001D1237C13B185F800B05BE0354B5C7B59
:10B40000002C08BF5A73394C6478002C52D0364C4B
:10B41000647814F0010F1EBFBF7B002FBAF5BA5F2E
:10B420000DD919F0400F01D0502E08D90A700678B6
:10B43000761CF6B20670032E28BF85F800B02A4F9E
:10B44000244E14F0020F367B1CBF93F80E90B9F116
:10B45000000F11D093F80D90B1450DD84A7090F8B7
:10B46000019009F1010909F0FF0980F80190B9F193
:10B47000030F28BF85F800B014F0040F18D0164C45
:10B48000A47AACB15B7B9E4212D3BB7F002B14BF6E
:10B4900064234FF4966343450AD28A708278521C23
:10B4A000D2B200E006E08270032A28BF85F800B01F
:10B4B0000A780AB980F800C04A78002A08BF80F8E4
:10B4C00001C08978002908BF80F802C0BDE8F08F6C
:10B4D000C803002094030020FA0300205B00002032
:10B4E000690200202004002074030020940400203E
:10B4F000580000209002002030B5174D174C2878D6
:10B5000058B12089A080E080A08840F6AC5100228C
:10B51000884205D3A28222820EE0F8F785F9F3E78C
:10B52000218801EBC1018900B1FBF0F1A1824EF647
:10B530006021B1FBF0F02082B4F91000002809DD91
:10B54000B4F90E1000EB8000C901400091FBF0F04F
:10B55000A88030BDAA8030BD500400202004002007
:10B560002DE9F04706462C4885696988B14201D328
:10B5700028880CE0007F6FF0010101EB8002AA5ADD
:10B580006FF00308B24206D808EB8000285ABDE8E5
:10B59000F04700F0EDBC0124022738E007EB8402FD
:10B5A000AA5AB24231D901EB8400285A00F0E0FCDB
:10B5B000814608EB8400285A00F0DAFC804607EB4D
:10B5C0008400285A00F0D4FC074635F8240000F027
:10B5D000CFFC04464946384600F0AAFD05464146E0
:10B5E000204600F0A5FD0446304600F0C1FC494667
:10B5F00000F09EFD214600F0CFFC294600F0D6FB6E
:10B600004146BDE8F04700F06FBB641CE4B2A042C5
:10B61000C4D80248BDE8F087680400200000C84292
:10B620002DE9F041DFF8ACC00424069D8CF80840F9
:10B63000294E00248CF80940778896F800E03F04F2
:10B64000767807EB0E273E44CCF8046008268CF889
:10B650000A60ACF16006EFB246F86B4F74608C1C68
:10B660002E0A04F03F040CF10E0522B1012A0CD081
:10B67000022A28D116E08CF80B400AE018B30529FD
:10B680000ED80A46014628461BE044F040028CF8DA
:10B690000B208CF80C708CF80D600029EED112E0B4
:10B6A0000521EEE703F00F0242F080028CF80B2038
:10B6B00049B140B1072900D907210A46014605488A
:10B6C0000C30F7F718FEBDE8F04102490348F8F7DF
:10B6D00014BB0000740500204000002000640040FE
:10B6E00070B51D4614460646402A00D9402422461D
:10B6F0000848F7F700FE0748A0F1880108608C8031
:10B70000CE800020088188720120C87202484570EE
:10B7100070BD00009C0500204000002002494FF051
:10B72000000000F07ABD00BF0000F87F2DE9C041A5
:10B7300030B4DFF8A0C23CEA111418BF3CEA13147D
:10B7400000F0EC8081EA03051CEA111444EAD57488
:10B7500018BF1CEA131500F0C780A4EB05044FF0D6
:10B76000004545EAC12145EAC32341EA505143EA75
:10B77000525304F17F74994204F500344FEAC0201B
:10B780004FEAC22208BF904200F09C804FEA136546
:10B790000FF24016765D4FEA134506FB05F7C7F139
:10B7A000807706FB07F74FEAD737A7FB0368764297
:10B7B000C8F58038A7FB06CE38BFA8F1010807FB03
:10B7C00008E64FF0000EA6FB028CE6FB03CEDCF190
:10B7D000000CCEF1004E38BFAEF1010EA6FB0C58A6
:10B7E0004FF000074FF00005E6FB0E87A1FB08C6EF
:10B7F000A0FB07CE16EB0E0645F10005E1FB076541
:10B8000015F1E04E7EBFA4F580345FEA46066D4137
:10B8100016F1800745F100054FEA17274FEA066643
:10B8200047EA0567A6F1DE46B6F1805F4FEA1525C7
:10B830001FD9384624F0010C05EBC471BCF1FE6F32
:10B8400001EB0C1102D8F0BCBDE8008124425CBFC2
:10B8500001F5801E9EEAC47F02D4F0BCBDE80081E1
:10B86000244238D4F0BCA1F1C041BDE8004100F051
:10B8700035BA4FEAD22242EA43524FEAD323A7FB1A
:10B8800002864FEAD02040EA415007FB03661EEAD9
:10B890000E0F4FEAD12105FB026658BFA6EB0056FA
:10B8A000B6EB00564FEA520E4EEAC37E18EB0E0E70
:10B8B00056EB530EBDD518EB02085E417F1C55F1C7
:10B8C0000005B6E74FF480154FF000074FF0000673
:10B8D0004FF00008ADE7F0BC4FF0000001F1C041AF
:10B8E00001F00041BDE8008111EA0C1F0CEA1315BC
:10B8F00000D00CE013EA0C1F00F025804FF0000090
:10B90000F0BC81EA030101F00041BDE80081F0BC18
:10B91000BDE8004181EA030100F0E0B9F0BCBDE8F8
:10B92000004170B500F08CF9097EFC3E00F007B8CC
:10B9300081EA03014FF0000001F00041704781EA05
:10B94000030100F0CBB9F0BCBDE800414FF00000AE
:10B9500021497047FFFDFBF9F7F5F4F2F0EEEDEB4E
:10B96000E9E8E6E4E3E1E0DEDDDBDAD8D7D5D4D3FD
:10B97000D1D0CFCDCCCBCAC8C7C6C5C4C2C1C0BF49
:10B98000BEBDBCBBBAB9B8B7B6B5B4B3B2B1B0AF4F
:10B99000AEADACABAAA9A8A8A7A6A5A4A3A3A2A133
:10B9A000A09F9F9E9D9C9C9B9A99999897979695EE
:10B9B00095949393929191908F8F8E8E8D8C8C8B8A
:10B9C0008B8A898988888787868585848483838212
:10B9D000828181800000FF070000F87F4FEA410369
:10B9E0004FEA5353A3F58063D3F11E03C8BFD3F1CD
:10B9F000210C0CDD4FF0004242EAC12242EA5052D3
:10BA000032FA03FC8CEAE17CACEBE1707047102B5E
:10BA1000C4BF0020704703F5787CBCF1FF3F04D021
:10BA20006FF0004282EA2100704770B500F008F91B
:10BA30004992248000207047F2E700004FEA11533A
:10BA4000A3F58063D3F11E03A8BFD3F1200C08DB5C
:10BA50004FF0004242EAC12252EA505232FA03F059
:10BA6000704709420BD4102BC4BF0020704703F568
:10BA7000787CBCF1FF3F05D04FF0FF3070474FF0AE
:10BA80000000704770B500F0DBF800BF49922480D9
:10BA900000207047F0E710F0004248BF4042B0FA83
:10BAA00080F310FA03F10AD0C3F11D0303F580639C
:10BAB0004FEA415002EB035202EBD12170474FF0A5
:10BAC00000007047B0FA80F310FA03F10AD0C3F116
:10BAD0001D0303F580634FEA41504FEA035202EB26
:10BAE000D12170474FF0000070470000DFF848C1D7
:10BAF00070B51CEA111E1EBF1CEA13159EEA0C0F3E
:10BB000095EA0C0F00F06F8081EA030423EA4C13DE
:10BB10004EEAD47E21EA4C1141F4801143F48013A3
:10BB2000AE44A1FB024CA0FB0365AEF17F7E36194B
:10BB300055EB0C05A1FB034C4CF10003A0FB021CD0
:10BB400016EB0C06654153F10003094218BF46F09D
:10BB5000010613F4007F0BD14FEA03314FEA0530A1
:10BB6000340341EA155140EA16506FF003020AE02F
:10BB70004FEAC3214FEAC520F40241EA555140EA99
:10BB800056506FF0020202EB2E4201EB025585EA9D
:10BB9000CE710AD05FEA440C18BF24F0004450F183
:10BBA000000041F1000120EAD47040F2FE7C6245C1
:10BBB00000D270BDA84214BF4FF080444FF0404403
:10BBC000002E08BF0024BEF1806FA8BFA1F1C041C4
:10BBD000BDE8704080F282804FF0000001F1C0416A
:10BBE00001F0004170479EEA0C0F0CEA131518BFD4
:10BBF00095EA0C0F06D04FF0000081EA030E0EF01C
:10BC0000004170BD00F01CF88900013E00F007B84B
:10BC100000F009B84FEA430C5FEA5C5C08D081EAA7
:10BC2000030100F05BB84FEA410C5FEA5C5CF6D1BF
:10BC30004FF00000014970470000FF070000F87F47
:10BC40000EF1020E2EF0030E5EF8046B364205D4A0
:10BC5000012A43EB030515F5001F12D8012841EB1B
:10BC6000010C1CF5001F0CD80ED14FEAD17C15F544
:10BC7000001F0CEB4C0C0CF1020C08BF4CEBD37CFE
:10BC800004E04FF0080C01E04FEAD37C0CEB4C05CC
:10BC900026FA05F606F00706B6F1040C06D20EEBFE
:10BCA000860CBDE870404CF0010C6047DFE80CF0FA
:10BCB000090B02024FF000414FF00000A1F50021F6
:10BCC00070BD19461046012851EB010418BFD4F588
:10BCD000001484BF002001F0004170BD0808A0F5E9
:10BCE00000114FEA3101704790EA010F48BF81F01F
:10BCF000004100F12482421A3CBF801A89184FEAA1
:10BD0000D0524FF07F4C1CEA410FA2EBD15318BF29
:10BD10009CEA026F00F03B804FF0004C4CEA0020A0
:10BD20004CEA012121FA03FC10EB0C0C1ED202F1AB
:10BD3000FF325FEA1C2040EBC25038BF70471CF056
:10BD40007F0F4FEA400C18BFBCF17F4F38BF7047E0
:10BD5000C3F12003994008BF20F00100BCF17F4FE0
:10BD600038BF7047A0F1C04000F0DDB94FEA3C0099
:10BD7000000A40EBC25028BF1CF0FF0F4FEA400CF6
:10BD8000E6D018BFBCF17F4F38BF7047EAE79CEAA6
:10BD9000026F05D010EA5C0F08BF00F0004070474A
:10BDA00010B500F07AF900BF64FBBE3E4FF47F0C83
:10BDB0001CEAD0121EBF1CEAD11392EA0C0F93EAC0
:10BDC0000C0F00F0858090EA010F48BF42F48072AA
:10BDD00040F4000C41F400002CF07F4120F07F4043
:10BDE00000B58142A2EB03020FF2081CACEB504EEF
:10BDF000C0F100009EF800E04FEA4E0E00FB0EFC82
:10BE000038BF49004FEA2C1C02F5FA020CFB0EF376
:10BE10004FEACE1E4FEA112C4FEAC1210EEB635EB2
:10BE200042EB22420EFB0CFC4FEA1C5300FB0311B9
:10BE30004FEA112C4FEA01310EFB0CFC4FEADC4CAF
:10BE400000FB0C11C14228BF09184CEB03335DF80D
:10BE500004EB10EB410143EBC250B2F57C0F38BF4D
:10BE6000704729D512F0F00F1CBF00F1C04000F060
:10BE700000407047008182838485868788898B8C07
:10BE80008D8E8F919293959697999A9C9D9FA0A243
:10BE9000A3A5A7A8AAACAEB0B2B3B5B7B9BCBEC093
:10BEA000C2C5C7C9CCCED1D4D7D9DCDFE2E6E9EC34
:10BEB000F0F3F7FAFE0000004FEA400C0CF1807C32
:10BEC000BCF17E4F28BF7047B0F1C04000F02BB9E5
:10BED00090EA010F0CEAD11348BF42F48072624528
:10BEE00038BF634507D213F47F0F16D080EA0100F4
:10BEF00000F00040704710B500F0CFF8097EFC3E1E
:10BF000000F005B880EA010000F00040704780EAC8
:10BF1000010000F0004000F006B912F47F0F04BFEA
:10BF20000248704780EA010000F0FDB80000C07FC1
:10BF3000C10DD1F19E0206DB4FEA002343F000431E
:10BF400023FA02F07047004207D54FEA4001B1F1F1
:10BF5000FE4F02D24FF00000704710B500F09DF880
:10BF600049922480002070476FEA2000704700004B
:10BF7000B0FA80F310FA03F2C3F19D030AD0D90599
:10BF800001EB1220530638BF704700F1010008BFD3
:10BF900020F00100704700004FF47F0C1CEAD01223
:10BFA0001EBF1CEAD11392EA0C0F93EA0C0F00F0AB
:10BFB000478090EA010F48BF42F480724FF0004C76
:10BFC0004CEA00204CEA012102EB0302A0FB011322
:10BFD000A2F50002002918BF43F001035B0028BF4F
:10BFE0004FEA330342EB22425FEA132C4CEBC25080
:10BFF0002EBFBCEB436FB2F57C0F70474FEA036C6A
:10C00000BCF1004F08BF20F00100B2F57C0F38BF33
:10C0100070470BD582F0FF0212F5803FC8BF704712
:10C0200000F1C040D8BF00F00040704700F5000CA0
:10C030005FEA4C0C48BF7047B0F1C04000F073B8E5
:10C0400090EA010F0CEAD11348BF42F480726245B6
:10C0500038BF634504D280EA010000F00040704719
:10C0600010B500F01AF800BF8900013E00F007B8D3
:10C0700000F009B85FEA410C5FEA1C6C08D080EA66
:10C08000010000F050B85FEA400C5FEA1C6CF6D18A
:10C090004FF00040A0F5800070470EF1020E2EF028
:10C0A000030E5EF8044B244204D44FEA4102B2F17D
:10C0B0007F4F11D84FEA4003B3F17F4F0CD80ED118
:10C0C0004FEAD07CB2F17F4F0CEB4C0C0CF1020C20
:10C0D00008BF4CEBD17C04E04FF0080C01E04FEAC4
:10C0E000D17C0CEB4C0324FA03F404F00704B4F104
:10C0F000040C06D20EEB840CBDE810404CF0010C91
:10C100006047DFE80CF0070802024FF00040A0F59E
:10C11000800010BD0846420018BFD2F1807288BF6F
:10C1200000F0004010BDFF2141EAD050C00570472B
:10C1300090EA010F48BF81F000413FF5DCAD421AA3
:10C1400004D882F00042A0EB020011444FEAD05222
:10C150004FF07F4C1CEA410FA2EBD15318BF9CEA71
:10C16000026F4AD04FF0004C4CEA00204CEA01210B
:10C1700021FA03FCB0EB0C0C0FD412F0FE0F36D0FA
:10C180005FEA4C001DD5001240EBC25038BF70472B
:10C190001CF03F0F18BF70470BE0A2F101025FEAED
:10C1A0001C2040EBC25038BF70471CF07F0F18BFF7
:10C1B0007047C3F12003994014BF401E20F00100D6
:10C1C000704780084FEA122308BF7047B0FA80FC1E
:10C1D000A2EB0C02CCF1280C60FA0CF093EA122FBF
:10C1E00004BF00EBC25070474FEAC3707047130A98
:10C1F0005FEADC1008BF7047F6E79CEA026F04D0E4
:10C2000010EA5C0F08BF0020704710B5FFF745FF2C
:10C2100040DFF63E81F0004070470CF00F03092B21
:10C2200008BF082000F059800A2B0BD0082B18BF3C
:10C23000704708BF1CF0400F0AD04FF000004FF0CD
:10C24000000170471CF0400F18BF4FF000407047CE
:10C250001CF0100F08D020F0704300F07F4242EA3B
:10C26000D3014FEA4370704700F0604021F07F42F5
:10C2700042EA000201F07F4040EA727070474FF0DE
:10C28000FF0C4CF4E06C1CEA11531CBF9CEA030C3D
:10C290009445C2BFDA4201EB02517047002B0DD02A
:10C2A000BCF1000F0FD0002A01F00041A4BF41F003
:10C2B000E04141F07F614FF00000704701F0004124
:10C2C0004FF00000704750EA01334FF09B0C18BF4D
:10C2D0004CF0806C7FF422AA70471CF4801F11D0B0
:10C2E0001CF4E02F03D06FEACC31490070474FF0C7
:10C2F0004050EFF3008222F0704242EA000282F3E3
:10C30000008870474FF000007047010002010000F4
:10C3100002000401020003000401060004001800EA
:10C320000A0005000A012200070002002C0000019B
:10C3300002002E0002010200300003010200320060
:10C340000D01040134001001040038001101040142
:10C350003C001F010401400060010401440010077B
:10C3600002014800110702014A00001102014C00BD
:10C37000021102014E0006F10A01970005F10400C6
:10C38000A10007F10400A50024010200A90004FF98
:10C390000100AB0059010201AC000019020052007B
:10C3A00025020400AE0020020200B40006010200D3
:10C3B000B20021020200B60023020400B8005701B7
:10C3C00015005300580115006800140118007D0085
:10C3D0000B09020195001318020150001209020115
:10C3E000BC0011090201BE0019010200C6001D189F
:10C3F0000401C8001E180401CC001A010200C40088
:10C4000013010201C00007F50200C2002019020159
:10C41000D0000000E8080500060908004C090A00E1
:10C420007409140092091E00C4092800D8093200BA
:10C43000000A3C00460A4B008C0A5A00D20A6400EB
:10C44000220B0000B20C0500E40C0800480D0A00A5
:10C450007A0D1400AC0D1E00E80D2800100E3200FD
:10C46000420E3C00A60E4B000A0F5A006E0F6400ED
:10C47000041000003C0F0500780F0800F00F0A00C0
:10C480002C10140068101E00B8102800E0103200B4
:10C490001C113C0094114B000C125A0084126400D1
:10C4A000F21200003610050068100800FE100A00A5
:10C4B000C6111400F8111E00481228008E12320016
:10C4C000CA123C0056134B00CE135A001E146400CF
:10C4D0008214000094110500D011080048120A00CF
:10C4E0008E121400D4121E0024132800561332009A
:10C4F0009C133C001E144B00A0145A001815640035
:10C500007C15000050140500A01408002C150A002A
:10C510007C151400CC151E0030162800761632004B
:10C52000C6163C005C174B00E8175A006A186400F6
:10C53000CE1800006A180500CE18080078190A0005
:10C54000DC191400401A1E00B81A2800081B32001B
:10C550006C1B3C00201C4B00D41C5A007E1D640048
:10C56000141E00000000C90092015B022403ED03C9
:10C57000B6047F0548061107D907A2086B09330ADC
:10C58000FB0AC40B8C0C540D1C0EE40EAB0F731085
:10C590003A110112C8128F1355141C15E215A81672
:10C5A0006E173318F918BE19831A471B0C1CD01CC0
:10C5B000931D571E1A1FDD1F9F2062212422E52292
:10C5C000A72367242825E825A82668272728E52803
:10C5D000A429622A1F2BDC2B992C552D112ECC2E31
:10C5E000872F4230FC30B5316E322733DF3397343A
:10C5F0004E350436BA3670372538D9388D39403A39
:10C60000F33AA53B573C083DB83D683E173FC63F4F
:10C6100074402141CE417A422643D1437B44244594
:10C62000CD4575461D47C4476A480F49B449584A25
:10C63000FB4A9E4B404CE14C814D214EC04E5E4F1B
:10C64000FB4F98503451CF51695203539B5333548D
:10C65000CA546055F6558A561E57B1574358D45898
:10C660006459F459825A105B9D5B295CB45C3E5D51
:10C67000C85D505ED75E5E5FE45F6860EC606F61CE
:10C68000F1617262F2627163EF636C64E964646524
:10C69000DE655766D0664767BD673268A7681A6966
:10C6A0008C69FD696E6ADD6A4B6BB86B246C8F6CAC
:10C6B000F96C626DCA6D316E976EFB6E5F6FC26F03
:10C6C00023708370E37041719E71FA715572AF727D
:10C6D00008735F73B6730B746074B3740575567525
:10C6E000A675F47542768E76D97623776C77B47713
:10C6F000FB7740788578C8780A794A798A79C97948
:10C70000067A427A7D7AB77AEF7A277B5D7B927BD5
:10C71000C67BF97B2A7C5A7C897CB77CE47C0F7DC4
:10C720003A7D637D8A7DB17DD67DFB7D1E7E3F7E19
:10C73000607E7F7E9D7EBA7ED67EF07E0A7F227FDF
:10C74000387F4E7F627F757F877F987FA77FB57F19
:10C75000C27FCE7FD97FE27FEA7FF17FF67FFA7FCB
:10C76000FE7FFF7FF8790000A27900004879000081
:10C77000EA7800008878000022780000B87700008E
:10C7800049770000D67600005E760000E175000073
:10C7900060750000DA7400004F740000BE73000082
:10C7A000297300008F720000EF7100004A710000D1
:10C7B000A0700000F06F00003B6F0000806E000072
:10C7C000C06D0000FA6C00002F6C00005F6B000071
:10C7D000896A0000AD690000CD680000E7670000CD
:10C7E000FB6600000B660000156500001B6400007E
:10C7F0001C630000186200000F610000026000006E
:10C80000F15E0000DC5D0000C35C0000A65B000080
:10C81000855A0000615900003A5800001057000086
:10C82000E3550000B4540000825300004F52000052
:10C830001A510000E34F0000AB4E0000724D0000A3
:10C84000384C0000FE4A0000C34900008848000040
:10C850004E47000014460000DA440000A2430000E6
:10C860006A4200003441000000400000CD3E00005C
:10C870009C3D00006D3C0000413B0000173A000069
:10C88000F0380000CB370000AA3600008B350000DE
:10C89000703400005833000044320000333100008F
:10C8A000263000001D2F0000172E0000162D00005E
:10C8B000182C00001F2B0000292A00003829000036
:10C8C0004A280000612700007C2600009B2500000C
:10C8D000BF240000E62300001223000041220000D4
:10C8E00075210000AD200000EA1F00002A1F000093
:10C8F0006E1E0000B71D0000031D0000531C000049
:10C90000A71B0000FF1A00005A1A0000BA19000005
:10C910001D19000083180000EE1700005B170000CF
:10C92000CC16000041160000B915000034150000B7
:10C93000B214000033140000B81300003F130000CD
:10C94000C912000057120000E71100007A11000020
:10C950000F110000A710000042100000E00F0000BF
:10C96000800F0000220F0000C60E00006D0E0000B8
:10C97000160E0000C20D00006F0D00001F0D00001C
:10C98000D00C0000840C0000390C0000F10B0000FA
:10C99000AA0B0000650B0000220B0000E00A00005B
:10C9A000A00A0000620A0000250A0000EA0900004F
:10C9B000B109000079090000420900000D090000DA
:10C9C000D8080000A6080000740800004408000011
:10C9D00015080000E7070000BB0700008F070000F4
:10C9E000650700003B0700000A7C0000E07B0000B8
:10C9F000AE7B00007A7B0000437B00000A7B0000D6
:10CA0000CF7A0000927A0000527A00000F7A00007C
:10CA1000BC7900008279000038790000EB780000D2
:10CA20009A78000047780000F177000098770000BE
:10CA30003B770000DC76000079760000127600007B
:10CA4000A87500003B750000CA7400005674000011
:10CA5000DE73000062730000E27200005F7200008B
:10CA6000D87100004D710000BE7000002B700000F6
:10CA7000946F0000FA6E00005B6E0000B86D00005D
:10CA8000126D0000676C0000B86B0000056B0000C1
:10CA90004F6A000094690000D66800001368000027
:10CAA0004D67000082660000B4650000E36400008A
:10CAB0000D640000346300005862000078610000DB
:10CAC00094600000AD5F0000C35E0000D65D000012
:10CAD000E65C0000F25B0000FC5A0000045A000013
:10CAE000085900000A5800000A57000008560000C4
:10CAF00003550000FC530000F4520000E95100000F
:10CB0000DE500000D14F0000C24E0000B34D0000C7
:10CB1000A34C0000914B00007F4A00006D490000CB
:10CB20005A480000474700003546000021450000F4
:10CB30000F440000FD420000EC41000019400000DD
:10CB4000CB3F0000BB3E0000AD3D0000A13C00001B
:10CB5000953B00008C3A0000843900007E380000CC
:10CB60007A37000077360000773500007A3400000D
:10CB70007E33000085320000D83000009A3000007B
:10CB8000A92F0000BB2E0000D02D0000E62C0000D5
:10CB9000012C00001F2B00003F2A0000612900002B
:10CBA00089280000B2270000DF26000011260000BF
:10CBB000452500007A240000B5230000F322000080
:10CBC0003422000079210000BF2000000A2000006C
:10CBD0005A1F0000AB1E0000001E0000591D00007F
:10CBE000B51C0000121C0000761B0000DB1A0000C0
:10CBF000431A0000AD1900001C1900008F18000036
:10CC0000031800007B170000F516000072160000E4
:10CC1000F215000076150000FD14000086140000D7
:10CC2000121400009F13000030130000C312000014
:10CC30005A120000F21100008C1100002A110000AD
:10CC4000CA100000691000000F100000B50F0000AE
:10CC50005C0F0000060F0000B40E0000610E000023
:10CC6000110E0000C30D0000770D00000808080831
:10CC7000080808080808000098CC000800000020F8
:10CC8000900200002831000818CD00089002002012
:10CC900088160000843100081184D8B80500092CDA
:10CCA0000102030406070809120103269C1C022D39
:10CCB00046EBFFFF10091C016102496E32065A075C
:10CCC000045A0510E908291CE928290469100912E9
:10CCD000346920E9280110032001010318CF0388DB
:10CCE000099E07DA16B42DDA160201160C17B0CA1F
:10CCF0000B66180807030602050104A910090301C1
:10CD00000604020706041B05020B140601050C129B
:08CD1000030204B30145000019
:04000005080030EDD2
:00000001FF
